:020000040800F2
:10500000181B0020D5500008898C00086183000817
:105010000000000000000000000000000000000090
:105020000000000000000000000000006999000876
:10503000000000000000000029920008819A00088A
:10504000E7500008E7500008E7500008E750000864
:10505000E7500008895D0008E7500008E7500008A5
:1050600000000000E7500008B15C0008E7500008AD
:10507000E75000087988000800000000E7500008A9
:1050800000000000E75000080000000000000000E1
:10509000E750000800000000E7500008E750000853
:1050A000E7500008E7500008E75000080DA5000889
:1050B000E7500008E7500008000000000000000072
:1050C0000348854600F040FD004800478DB80008C1
:1050D000181B00200448804704480047FEE7FEE70D
:1050E000FEE7FEE7FEE7FEE71D9B0008C150000853
:1050F00030B50B46014600202022012409E00D4670
:10510000D5409D4205D31D469540491B25469540F7
:1051100040191546521E002DF1DC30BDF0B51FB40C
:105120000646002082B005464024019100901BE015
:10513000019922460F46304600F0F0FB049A059B89
:10514000801A994110D310461946224600F0D6FB2A
:10515000361A8F410197224601200021009F00F05E
:10516000CDFB38184D4100902046641E0028DFDC3E
:10517000019B00982946324607B0F0BD03460B4319
:105180009B0703D009E008C9121F08C0042AFAD2FD
:1051900003E00B780370401C491C521EF9D2704783
:1051A000D2B201E00270401C491EFBD270470022BF
:1051B000F6E710B513460A4604461946FFF7F0FF16
:1051C000204610BD30B504460020034600E05B1CBD
:1051D000934203D2E05CCD5C401BF8D030BDF8B503
:1051E00002464A40D40F42004B0052085B089A42E4
:1051F00002D20246084611464A0023D0C30D4A0097
:10520000DDB2120EAD1A202D35DA49020126490A07
:10521000F6058A19002C00D0524220214F1B11465E
:10522000B9402A411018C20D9A4221D0002C17D043
:10523000012D08DCDA05801AD20F8019D207DBB203
:1052400000F098FBF8BDDA05801A012340001B0628
:10525000C01880185A428018CA0F1043490007E04E
:105260004908C2071143DA05801A801940088018DE
:1052700000F078FBF8BD61000122511A001BF7E72E
:105280000122D2075140AAE70122D2075040A6E7E7
:10529000024670B54A40D30FDB0740002DD04A00CC
:1052A0002AD0010E140E000212020919400A520AF5
:1052B0008418E50104465443000A120A2E045043A0
:1052C000A4194219200CC543AA18120C0125AD03DC
:1052D000521C521912047F39240400D0521C10436E
:1052E00001D44000491EC2B20C06C0092018401C5F
:1052F0004008802A02D003E0002070BD4008400032
:10530000002900DA0020184370BD70B502464A40FB
:10531000D50F40004A00ED0740085208002814D07D
:10532000002A12D0C40DD30D41020120C005520243
:10533000490A520AE41A091812187D34914201D31D
:10534000641C00E04900002C01DA002070BD00233D
:10535000914201D3891A0343400849000028F7D13C
:1053600000290AD0914202D10121C90705E09142EA
:1053700001D2012101E00121C943E005C018401913
:1053800000F0F0FA70BD420005D04200120E524209
:105390008A4201DB00207047C905081870470000E9
:1053A000F0B507460846584087B0C00F0490480043
:1053B0000E46590040084908BC1A884105D23846B3
:1053C00031461E4617460B46024658004008104319
:1053D0004CD0300D039040055900400D490D05900B
:1053E000401A0290402872DA18030121000B0905C7
:1053F0000843019004980092002805D00199524278
:105400000020884100920190029840210A1A0199D7
:10541000009800F073FA05460C466B4607CB00F087
:105420008EFAC0197141039A0E0D0023D71756400A
:105430001A467A40164344D0049A002A2DD0029A84
:10544000012A039A15DC1205C01A9141012636057E
:10545000001C7141D20F059ED20700930192029663
:105460002A46234600F0CCFA07B0F0BD3846314654
:10547000FAE71605224A0F46B218C01AB7410121B1
:105480000905001C4F4100187F4111461818794149
:10549000E20F10436D19644113E0E2076D081543F4
:1054A0006408C2071443039A01261205C01A9141E9
:1054B0003605001C7141CE07400830434908C0182A
:1054C00051412A46234600F08EFACDE7FFE70498C3
:1054D00001224000C117121A00238B410498314663
:1054E000C417381AA141EEE730B40124E407634041
:1054F00030BC55E730B40124E407614030BC4FE7CD
:105500000000E0FFF0B51FB488B00B9909980024A3
:1055100048400999C00F490049080991C0070B99F3
:105520000090490049080B9109990898A64608433C
:105530001CD00B990A98084318D009980124400000
:10554000420D4800410D099824050003000B20433B
:1055500009900B980003000B20430B9050181C4936
:105560004018002201901446104605E00020014634
:105570000DB0F0BD032801DA034600E003239C468A
:10558000C11A0AAE0AE05F0008ADED5B4F00F75BA1
:105590007D430027AA187C41491C5B1E6145F2DD52
:1055A000410004AB5A522104120C0A43240C401C43
:1055B0000828DFDB01980290009970460191009065
:1055C000059B049A0799069800F01AFAD0E70000A4
:1055D0000DFCFFFFF0B50C465C4085B0E40FE4071E
:1055E00003944C000026640859009446490802467A
:1055F0000296224321D062460A431ED06200570D14
:105600004A000E032303550D012402462C492405AC
:10561000781B1B0B360B4018234326436146009032
:105620001C46501AB44103D30098401C009002E07D
:10563000921800985B41002803DA0020014605B06B
:10564000F0BD0020012109050746864611E06446A9
:105650001D46141BB54106D36546521BB341744623
:1056600007430C43A646CD07400849082843921833
:105670005B4105460D43EAD11046184313D06046FE
:10568000194650407140084306D06046101AB34195
:1056900006D20122002306E000220123DB0702E0FC
:1056A0000122D2435310009874460105381C614111
:1056B000029C039D0019694100F095F9BFE70000C5
:1056C000FD03000070B54B005B0803430BD04B009B
:1056D0005C0D002633466542B341D417AD1AA34191
:1056E00002DB0020014670BD12053018514170BD2B
:1056F000C217C10F504010B54018CA0796230021A9
:1057000000F038F910BD10B500229623114600F0C4
:1057100031F910BD0EB5C217C10F5040CA0740186D
:105720000021054B0293019200910A460B4600F0BE
:1057300067F903B000BD0000330400000EB5054951
:105740000291002100910A460B46019100F058F9A0
:1057500003B000BD33040000C20F4100400201232A
:10576000400ADB05D207090EC0187F2901DA0020A4
:105770007047962903DC9623591AC84001E09639F0
:105780008840002AF4D04042704741004002012284
:10579000400AD205090E80187F2901DA00207047DF
:1057A000962903DC9622511AC840704796398840E2
:1057B0007047000070B5CD0F4A0009030123090BA3
:1057C0001B0519430B4BED070024520D9A4201DAD9
:1057D000002070BD074B34339A4203DC9A1A00F064
:1057E0009DF802E00449511888402C43F1D0404212
:1057F00070BD0000FF030000CDFBFFFF4A0009035E
:105800000123090B1B051943094B10B5520D9A4290
:1058100001DA002010BD064B34339A4203DC9A1A99
:1058200000F07CF810BD03495118884010BD0000FD
:10583000FF030000CDFBFFFFC20FD207400040086E
:105840000BD0C10D0723DB01C91840020905400A2E
:105850001143C208400711437047002001467047BA
:1058600010B5002904DB0124E40740428C412146A5
:10587000002B04DB1C460123DB075242A3418B4271
:1058800000D1824210BD000010B5002904DB0124C4
:10589000E40740428C412146002B04DB1C460123D7
:1058A000DB075242A341994200D1904210BD000053
:1058B000CB0FDB07490010B5490802460A4307D061
:1058C0000A0D07240903E401090B121B002A01DC5D
:1058D000002010BDC900440F0C43C100E018D205E0
:1058E000801800F03FF810BD0122D207002800DB2D
:1058F000101A002900DB511A8142704710B5202A86
:1059000004DB0146203A9140002010BD9140202345
:105910009C1A0346E3401943904010BD10B5202A5D
:1059200004DB0846203AD040002110BD0B46D3408E
:10593000D0402024A21A91400843194610BD10B54A
:10594000202A06DBCB170846203A1041C1170B432B
:1059500006E00B461341D0402024A21A9140084390
:10596000194610BD002904DA401C490001D1400845
:105970004000704770B40024050C05D110240004C9
:1059800002D1002921D01124050E01D100020834D2
:10599000050F01D10001241D850F01D18000A41C39
:1059A000002801DB4000641C002908D020252E1BA4
:1059B0000D46F540A14000D00121294308430106CE
:1059C0001B1B000ADB1D02D5002070BC7047DB05E5
:1059D000181880180029F8DA401C4900F5D170BC6D
:1059E00040084000704710B5002B08DA0024401C26
:1059F000614192185B411A4301D14008400010BD3B
:105A0000F0B51FB482B005460C0003D0084604F080
:105A100037FE02E004F034FE2030024600902146BA
:105A20002846FFF76BFF049B059A04460F46184370
:105A30001143084314D0184610431BD0009840214E
:105A40000A1A18460599FFF769FF05460E46009A9F
:105A500005990498FFF752FF084305D0012004E0A0
:105A60002046394607B0F0BD0020C11705430E435C
:105A70002C43374300990E986305401A7905E40AD0
:105A800000220C43FD0A0A3002D500200146E9E756
:105A90000105101969410C9C0D9D00196941FFF722
:105AA000A2FFDFE7FEB500231A461B1A8A4103DB7B
:105AB0000020014603B0F0BD4A000D0301212D0B6B
:105AC0000905520D0D43D10702D100186D41521E38
:105AD0005110FF31FF310131002704463E46384660
:105AE000009701910246012100200905FFF716FFEA
:105AF000C3197141F818324684468E464A416146C0
:105B00002846611A904104D36046241A954176468E
:105B10001F46241900986D41401C00903428E1DD97
:105B2000F91930467041091BA84103D20022D24323
:105B3000134601E00022134601980105381C71410B
:105B4000FFF751FFB6E70000064C0125064E05E0C1
:105B5000E36807CC2B430C3C98471034B442F7D38E
:105B6000FFF7B2FA80C70008A0C7000870B58C180C
:105B70000578401C6B075B0F01D10378401C2A118C
:105B800006D10278401C03E006780E70401C491CC8
:105B90005B1EF9D12B0705D40023521E0DD40B70C8
:105BA000491CFAE70378401CCB1A921C03E01D78CD
:105BB0000D70491C5B1C521EF9D5A142D8D30020A0
:105BC00070BD000038B50446064805490068FFF777
:105BD0008FFA604300E0401E00900028FBD138BDE2
:105BE00040420F005C010020F8B50446006881685F
:105BF0008907890F012902D10168C90722D181686B
:105C0000114A10261140012500290ED1816829432F
:105C100081600120FFF7D6FF01F006F807460CE08F
:105C200001F002F8C01B0A2807D9606D3043606597
:105C3000A06D2843A0650120F8BD20680068C0431E
:105C4000C007EDD10020F8BD170000801FB50B483C
:105C500000900B4801900B4802900B480390694656
:105C60000A4805F003F90A4A08481146083904F0C1
:105C7000EBFF00F04DFA002004B010BD89C500080C
:105C800065C50008C5C50008C3C500086801002037
:105C90001000002010B500231A4603E0845CE318CE
:105CA0009BB2521C8A42F9D3D84380B210BD000087
:105CB00010B5034800F074FD024800F071FD10BDFE
:105CC000B41600206C16002030B5446C1C252C4006
:105CD0000125A540046C6560046863608368102B2F
:105CE000036803D099600068C26030BD9A600068A4
:105CF000C16030BD1449012048720A4602205E325C
:105D0000507203203C3A507204200E3A50720F48F1
:105D10000D4B0078087022310870203108770C494B
:105D20005A1C087858714978997123331871597140
:105D3000203318775977107551751A461E32107531
:105D40005175107651767047C01100200B0100206C
:105D50002C01002010B503F0DDFD202003F086FEAD
:105D6000012005F0EDFA002003F080FE044805F064
:105D70008BF9044805F03AFC002005F06FFC10BDDB
:105D8000E000002083800000F8B505200121000715
:105D900000F036FF0025174C002800D06560164E35
:105DA0000221304600F02CFF00281BD1012020707A
:105DB0001248808F00280ED00127BF0200223946EA
:105DC000304600F02AFF0A2004F0AEFE01223946D8
:105DD000304600F022FF0A48656000880A214843E7
:105DE00008490880012000F043FE022000F040FE38
:105DF000F8BD00004801002000040050C00D002044
:105E0000180100202A0100207047000010B5084941
:105E100000224A6107494B684C1523434B604B688D
:105E2000082423434B60C009C001026010BD00007C
:105E3000FC160020002002407FB500250C460646D7
:105E4000039500F0E5FDE009029003A90196009595
:105E5000684600F075FD002804D000F0ADFD00207C
:105E600004B070BD00F0A8FD0120F9E710B50023D3
:105E700002E0C45CCC545B1C9342FAD310BD00001A
:105E800010B5214A00219069C305204804D5416915
:105E9000022319434161911593699B0505D5436917
:105EA0000124234343616302194393695B0505D5CC
:105EB0004369082423434361E301194393691B05A4
:105EC00005D543690424234343616302194393695D
:105ED0009B0405D54369102423434361630219439E
:105EE00093699B0304D5446920231C4344611943EF
:105EF0009369DB0305D54369402423434361A00232
:105F00000143916110BD000000200240FC160020FA
:105F100070B5054600F088FE0646184C0AE0681C7D
:105F200008D0002D04D000F07FFE801BA84201D9CC
:105F3000032070BDA069C007F1D1A069800701D519
:105F40000220A061A069C00511D4A06980050ED40B
:105F5000A06940050BD4A069000508D4A06980049D
:105F600005D4A069800302D4A069C00303D5FFF75C
:105F700087FF012070BD002070BD0000002002409E
:105F8000F8B51746002605460C4600F041FD09E02D
:105F900029460220226800F01DFD002804D1241D9E
:105FA0002D1D361DBE42F3D300F006FDBE4201D2C8
:105FB0000020F8BD0120F8BD10B5084902460020B8
:105FC000054B497905E044001C5B944203D0401C1A
:105FD000C0B28842F7D310BDE81200207000002044
:105FE00010B500F012FE10BD10B5094801F03CF8E4
:105FF00080B2FFF7A3FB074A074BFFF783FA0022A3
:10600000064BFFF7E7FAFFF7F9FB80B210BD00007F
:1060100020150020F853E3A59B843E4000408F40AC
:1060200070B5374C3548E083364821468A7F027583
:10603000C97F417534490A780276497841763149F9
:106040000520133148720A2005F0C0FA7D20C000F7
:1060500005F0D6FA2B49002213310C2005F0A0FBE5
:1060600000210C2005F0AEFB022005F0FFFA274DC1
:1060700000210F2005F02AFA28422063F8D0206B77
:10608000411C38D0400435D58122D20100210F2097
:1060900005F05BFB0021102005F018FA41061948B5
:1060A000490E0022633005F047FA164D6335687AD1
:1060B00005281FD102221449681DFFF783F8002824
:1060C00018D10F48AE7C66710422691C4830FFF776
:1060D00055F829461331084672000D465130FFF736
:1060E0004DF86079294642000648DF30FFF746F850
:1060F0000320207070BD04F037FB000024970000DF
:1061000070000020211200202C01002000D0272444
:1061100010B5144C1448224610321146083904F0C8
:1061200093FD0022114BE168A068FFF753FA104A73
:10613000104B05F0B9FC00220F4BFFF7DBF90022F2
:106140000E4BFFF7DFF9FFF7B3FB20600022134689
:10615000E168A068FFF784FB01D0206810BD002033
:10616000206010BD000000206801002000AA8F40C0
:106170006C45D9CC955BC83F0000F03F40A5E54099
:1061800010B5084800F096FA0A21064800F032FAE5
:10619000044800F01DF9800503D5024800F01AF903
:1061A00080B210BDC4140020F8B52F4D002201218B
:1061B000284600F032FDFFF7E3FFFFF7A4FA2B4E6D
:1061C0003146FFF7A2F82A4C0122A060114628466A
:1061D00000F023FD2749A068002588423EDB207897
:1061E000254F002815D02570FFF7CAFFFFF78BFA5F
:1061F0003146FFF78AF8A060FFF71EFB00223B46FE
:10620000FFF772F900221D4BFFF77CF9FFF750FBF7
:106210006060A068FFF710FB00223B46FFF764F9BF
:10622000174A184BFFF76EF906460F466068FFF7EE
:1062300003FB134A144B5242FFF764F932463B46C4
:10624000FFF7AEF8FFF734FB10496060884201DDCC
:10625000616004E0FF21C905C84200D36560606841
:10626000FFF793FAC0B2F8BD0004005000401B4491
:10627000480000200000604000000C4000E0644046
:106280003333333333B33040CCCCEC3F0000C8421F
:10629000F8B5054604464035287C0026012808D07C
:1062A00001202874206881688907890F01290ED18F
:1062B00001E00220F8BD0168C90708D0606D202107
:1062C000084360650126002028743046F8BD616DE2
:1062D000FF2201329143022211436165C16889079F
:1062E000890F0091C16889088900C16020688168B0
:1062F00092071143816000F097FC07460EE000F022
:1063000093FCC01B0A2809D9606D02218843102123
:1063100008436065002028740120F8BD206880686B
:106320000028ECDB2068C168009A1143C160606DF1
:1063300080088000401C6065C5E70000F8B506468F
:106340000D464036317C01290DD0012131740168A0
:106350008A68520709D5416D20221143416500200A
:1063600030740120F8BD0220F8BD174B6A68D805CB
:1063700047109A42154C8A6A2B6812D05B035B0B5C
:106380001A438A622968490305D5A1680143A160BF
:106390000A20FFF717FC2868800312D5A06838434D
:1063A0000EE05B035B0B9A438A622968490302D5BE
:1063B000A1688143A1602868800302D5A068B84322
:1063C000A06000203074F8BD0110000000270140DB
:1063D000406D70470068006C7047000070B50400A5
:1063E00006D0606D264600254036002802D006E023
:1063F000012070BDA5653574204600F0D3F8606DAE
:10640000C00603D421688868400705D5606D102157
:10641000084360653574EBE7606DFF2201329043FD
:1064200002221043606588688207920F5B48012A48
:1064300002D10A68D2072BD1032362689B079A42D4
:1064400005D05B429A4202D05B009A4209D10A69A8
:10645000920092080A6121680A6963681A430A6116
:106460000CE00A69920092080A6181680F22920486
:106470009143816081686268114381602168CA68C4
:1064800018239A43CA602168CA68A3681A43CA607D
:10649000816801225206914381608168A28E520672
:1064A0001143816020688168C90004D48168012299
:1064B0001207114381602068C168394A1140C160E8
:1064C0002069E168022825D00020014320462030C1
:1064D0000278037B52035B001A431143226B114382
:1064E000A26992031143E269D20311432268D3687F
:1064F0001943D160616A0A46FF3AC23A05D0A26ADE
:1065000011432268D3681943D16042780121012ADE
:1065100002D00BE00420D8E70078002823D0606D7B
:10652000202210436065A06D0843A065E06B012840
:1065300020681FD00169C90703D0016949084900D3
:10654000016120684169C908C90041612068416949
:10655000A26B11434161A565606D80088000401CFD
:106560006065002070BD2068C26801231B041A43C7
:10657000C260DBE70269FF239B009A430261206847
:106580000269236CA66C1A43636C33431A4302619D
:10659000206802690A430261D3E700000027014036
:1065A0001902FEFF10B586B0044614216846FEF7B6
:1065B000FEFD0E492068884216D10D48416B4215F8
:1065C00011434163C16A01221143C162C06A694635
:1065D00010400590022000900320019000200290BE
:1065E0000520000700F050FA06B010BD002401405D
:1065F00000100240F8B504464069254640350E4675
:1066000008280BD02068C068C00709D0606D202121
:1066100008436065002028740120F8BD082700E0C9
:106620000C2700F001FB009011E0701C0FD0002E31
:1066300005D000F0F9FA0099401AB04207D9606D10
:10664000042108436065002028740320F8BD2068F9
:1066500000683842E9D0606D012149020843606555
:106660002068C16809058A0F0C21002A1BD120224D
:10667000125D002A17D10268120714D582685307E9
:106680000122002B08DB43688B434360606D1302DB
:1066900098431043606506E0606D202318436065F1
:1066A000A06D1043A065A069002801D12068016099
:1066B0000020F8BD70B504462168002089684907AC
:1066C00021D425464035297C01291CD0012129747B
:1066D000E169012904D02046FFF786FA002811D18C
:1066E000616D0A4A1140FF220132114361650021A8
:1066F000A165297422681C21116021688A6804231D
:106700001A438A6070BD022070BD0000FEF1FFFFD9
:1067100030B5014620314A790023022A04D00422F0
:10672000C2630B71012030BD026814680E25AC43B2
:10673000146002681468640864001460446C1C22CD
:10674000144001221546006CA54045604A71184668
:106750000B7130BD70B50024014620314A79022A00
:1067600003D00421C163012418E0026813680E25D8
:10677000AB431360026813685B085B001360436CF3
:106780001C221340012215469D40036C5D604A7136
:1067900000220A71816B002900D08847204670BD15
:1067A000F0B4016C0D6801680C68466C1C2304226F
:1067B0001E401746B7402F420ED067070CD50C6815
:1067C000A40602D40C6894430C60416C19408A40C2
:1067D000016C4A60016B1AE00227B74002462F4065
:1067E0002032002F17D0A70715D50C68A40605D4B2
:1067F0000C680A25AC430C6001215171446C0221E4
:106800001C40036CA140596000211171C16A00292C
:1068100018D0F0BC08470827B7402F4212D02407F1
:1068200010D50C680E25AC430C60446C01211C4053
:106830000B46A340046C6360C16351710021117168
:10684000416BE4E7F0BC704770B504003CD01F48D2
:10685000256814212818FEF74BFC800060641C4852
:1068600020640221204620300246417129681948DF
:10687000E3680140A06866691843236933431843FD
:10688000A3691843E3691843236A1843084328603F
:106890000121A0688903884210D00D488030836AA6
:1068A000656C1C210D400F26AE40B3438362656CBE
:1068B00063680D40816AAB400B4383620020E06354
:1068C00001215171107170BD012070BDF8FFFDBF35
:1068D000000002400F80FFFFF8B504468C462030D0
:1068E00001790025012909D0012606714179002787
:1068F000012905D0077102252846F8BD0220F8BD00
:1069000002214171E763206801684908490001607C
:1069100061462046FFF7D8F9206B002820680168FF
:1069200001D00E2205E00422914301602068016835
:106930000A22114301602068016831430160DBE7EE
:10694000F8B51A4E0546307C0F46012807D00120C5
:1069500030741748FFF7DCFA010002D021E0022072
:10696000F8BD0020C04338606C6814E02046FFF793
:106970004DFA0F48FFF7CCFA01460E48426808234B
:106980009A434260426843159A434260002901D00D
:106990003C6006E08034A8686A68C0018018A042A4
:1069A000E4D8002030740846F8BD0000FC16002032
:1069B00050C30000002002400548416802221143F4
:1069C000416041680122114341600020704700008E
:1069D00000200240F8B50C4C1646207C0F460128DA
:1069E00008D0012020740948FFF792FA00250028FA
:1069F00002D006E00220F8BD65613E600348FFF763
:106A000087FA2574F8BD0000FC16002050C3000072
:106A100011484168C9070BD0EFF3108172B60F4AD5
:106A2000C2600F4AC26081F310884168C9070ED165
:106A3000416889070DD5EFF3108172B6094A0261EA
:106A4000094A026181F310884068800701D501205E
:106A5000704700207047000000200240EFCDAB8956
:106A600005040302BFAE9D8C161514137047000079
:106A700010B504494A69024202D04861FFF7F6FFA7
:106A800010BD000000040140FCB500230124A2E079
:106A900027462A469F403A406FD04D68012D05D0C9
:106AA000022D03D0112D01D0122D16D18568032699
:106AB000AC465D00AE46AE406546B543AC46CE68DA
:106AC0007546AE4065462E43866046680D79BE43E6
:106AD000ED06ED0F9D4035434560C6685F00032518
:106AE000BD40AE46AE4335468E68BE402E43C660BE
:106AF0004E68022E01D0122E14D1DE08B6003618D0
:106B00000196366A5D07B446EE0E0F25B540009635
:106B10006646AE43B4460D69009EB54066462E43B8
:106B2000019D2E6206687546AE430D79AD07AD0F27
:106B3000BD40354305604D68ED004BD5294D6E6B6A
:106B400026436E639E08284DB6007519AC46AD68A5
:106B50009E07360F0F27B740BD4305273F07B842B2
:106B600001D1002715E0214FB84201D1012710E0E3
:106B70001F4FB84202D102270BE02BE01D4FB84255
:106B800001D1032705E01C4FB84201D1052700E0E1
:106B90000627B7402F436546AF60184D2E684F68F3
:106BA0009643FF0300D516432E606E684F689643E8
:106BB000BF0300D516436E60AE684F689643FF0270
:106BC00000D51643AE60EE684F689643BF0200D50D
:106BD0001643EE605B1C0A681546DA4000D057E7A2
:106BE000FCBD000000100240000001400004005005
:106BF00000080050000C0050001C00500004014030
:106C00000069084000D001207047426913460B40DC
:106C10001B0491430B4383617047002A01D08161BB
:106C2000704781627047000001488068704700002B
:106C300050010020024881680278891881607047FD
:106C40005001002010B5084800240168402211437B
:106C50000160204600F00AF8002801D0012401E07C
:106C600000F04CFA204610BD0020024070B50446EA
:106C70000D4D7D202978C000FEF73AFA01460B48F9
:106C80000068FEF735FA00F035FF002809D1042C22
:106C900007D200222146401E00F058FA00206C6006
:106CA00070BD012070BD0000500100205C0100207B
:106CB00070477047F8B5654CA078401CA070012063
:106CC0002071A08B401CA0836148008802F08AFEDE
:106CD000208AFEF718FD01467F20C005FEF715FB50
:106CE0005C4D06462968FEF77AFA28600120A16A01
:106CF000C005814201DA084603E03046FEF7C4FAD7
:106D0000A062FF21C9050025C84200D3A5626078B2
:106D100000280BD102215048FFF772FF02004F49B3
:106D20004F4817D00022FFF778FFA56302214A4899
:106D3000FFF766FF4B4E002855D0A563B08AFEF7DB
:106D4000E2FC444F3968FEF7CFFD5FD2464901208F
:106D500008705DE00122D1034148FFF75EFF208A01
:106D6000FEF7D1FC01467F20C005FEF7CEFAA16BED
:106D7000FEF735FA3D49A0638842D7DD394801273F
:106D8000F926403000900A213046FEF7B1F900297B
:106D900003D132493248FFF723F902212E48FFF789
:106DA0002FFF002801D0002701E0002F12D102217F
:106DB0002948FFF725FF00280CD104F03DFE00997B
:106DC0000120888005F094FB642003F0ADFE294982
:106DD0002748C8600A2003F0A7FE3046761EF6B2A8
:106DE0000028D0D1A2E7208AFEF78DFC01467F2043
:106DF000C005FEF78AFAA16BFEF7F1F91E49A06300
:106E000088429BDB1B491A48C86097E71648057003
:106E1000708F401EFEF76CFC3968FEF765FD06D8E2
:106E20006079002803D015490120087001E013485B
:106E30000570708FFEF767FC3968FEF755FD04D2C8
:106E40006079002801D004F0BBFDF8BD08010020E6
:106E50008C0000204C010020000400500080000045
:106E600000000050C00D00207600002000004040CF
:106E70000400FA0500ED00E00000A04083000020BF
:106E8000704770B5040010D0022025462035A87345
:106E9000204601F0F9FCA87B032805D0204600F02D
:106EA000B9F80020A873687370BD012070BD7047E9
:106EB000704710B5044600680168C943C90708D186
:106EC0008168C943C90704D1012141602046FFF709
:106ED000F1FE20680168C943890708D48168C94365
:106EE000890704D4022141602046FFF7E1FE2068B3
:106EF0000168C943490708D48168C943490704D4D4
:106F000004214160204600F0F7F820680168C94379
:106F1000090708D48168C943090704D408214160DE
:106F20002046FFF7ADFF20680168C943C90608D4B1
:106F30008168C943C90604D4102141602046FFF787
:106F4000B8FE20680168C943890608D48168C9432E
:106F5000890604D4202141602046FFF7A9FF20685C
:106F60000168C943490608D48168C943490604D465
:106F7000402141602046FFF79AFF10BDF8B504009C
:106F800005D025462035A87B002802D006E0012048
:106F9000F8BD00206873204600F04EF80220A87368
:106FA0002068C26884466368012B01D106208243B1
:106FB00016486169814202D0072040038243002BBA
:106FC00001D1D82082431248A668024018463043B7
:106FD000676A266A3E433043A66A30431043002B5B
:106FE00002D0012B04D005E02369E2691A4300E0D6
:106FF000E2681043054A914202D0A2691143084356
:107000006146C8600120A8730020F8BDFFFF0000A2
:10701000F8F119FF10B500680549884207D1054805
:10702000816B4900490881630D2000F073F810BDA1
:10703000007C00400010024010B5006808498842FA
:107040000CD10848816BC2041143816300220121E5
:107050000D2000F07BF80D2000F06CF810BD000052
:10706000007C0040001002400068C06970470000CA
:10707000F8B504460220254620351746A8731D485A
:107080000268C3041A4302602068C2689B121A4354
:10709000C260206802690126324302612268102022
:1070A0005060206881611021204601F05DFC0328BA
:1070B0001FD02168082048602068476108212046C9
:1070C00001F052FC032814D0204601F0DDFBA87B20
:1070D00003280ED0206881683143816020680169EF
:1070E0003143016120680169042211430161AE73DB
:1070F0000020F8BD00040140704700000448416BC7
:10710000012211434163816B020411438163704783
:1071100000100240002809DBC106C90E012088408A
:1071200003490860BFF34F8FBFF36F8F70470000B4
:1071300080E100E0002805DBC106C90E012088407F
:10714000014908607047000000E100E010B503F05D
:10715000E9FA10BD02494A6882434A60704700005C
:1071600000700040024801688215114301607047B9
:107170000070004002494A6802434A6070470000BC
:107180000070004005480168022211430160044874
:10719000016904221143016130BF70470070004053
:1071A00000ED00E0F0B5154A1368154D54152D6A31
:1071B0002340ED07ED0F002B04D0002D02D0166800
:1071C000A64316601668B608B600064316600D485A
:1071D000076904263743076101290DD040BF20BF4E
:1071E00020BF0169B1430161002B04D0002D02D002
:1071F000106820431060F0BD30BFF2E7007000401F
:107200000000014000ED00E0F8B5044600780027DA
:10721000534D800671D5524E403EB06BC00004D431
:10722000B06BA9050843B06301274E480168C90542
:1072300011D40168821511430160FFF7F5FC00903D
:1072400005E0FFF7F1FC0099401A642837D845485B
:107250000068C005F5D532680321090560680A4059
:107260000140914208D08103890F032904D131687C
:10727000890301D50120F8BD2A69032109040A40C8
:1072800022D0084090421FD0207880061CD5286963
:107290002A6988430121C9040A432A612A698A4369
:1072A0002A612861C0050FD5FFF7BEFC009008E0F9
:1072B000FFF7BAFC0099411A2B48814201D90320FB
:1072C000F8BD28698005F3D561688803800F03281D
:1072D00005D132680005824301400A4332602869C3
:1072E000032261681204114008432861002F04D072
:1072F000B16B012000078143B1632078C00705D03E
:10730000E868A168800880000843E860207880076A
:1073100005D5E8680C218843E1680843E8602078D7
:10732000400706D5E868032189028843216908439C
:10733000E8602078000706D5E86803210903884340
:1073400061690843E8602078000606D5E8680321F3
:1073500089048843A1690843E8600020F8BD000063
:10736000401002400070004088130000F8B50E463F
:10737000050038D05E480068C007C00FB04214D284
:107380005B4C20684008400030432060FFF74CFC15
:10739000074605E0FFF748FCC11B564881427AD8F2
:1073A0002068C007C00FB042F4D12878524C800743
:1073B00005D5E068F0218843A9680843E060287893
:1073C000C00752D06868022806D0032807D0216879
:1073D00001280AD0890504E02168890301E02168B9
:1073E0008901002903DB0120F8BD4907F9E7E168BD
:1073F000890889000143E160FFF716FC07466868C9
:1074000002280AD0032814D001281ED029E0FFF753
:107410000BFCC11B374881423DD8E0680007800F54
:107420000228F4D121E0FFF7FFFBC11B3148814264
:1074300031D8E0680007800F0328F4D115E0FFF78A
:10744000F3FBC11B2B48814225D8E0680007800F61
:107450000128F4D109E0FFF7E7FBC11B2548814271
:1074600019D8E0680007800FF5D121480168C907E5
:10747000C90FB14217D90168490849003143016079
:10748000FFF7D2FB074608E005E0FFF7CDFBC11B85
:107490001848814201D90320F8BD15480068C0078B
:1074A000C00FB042F1D12878400706D5E068072127
:1074B00009028843E9680843E0602878000707D597
:1074C000E0680721C90288432969C9000843E060D0
:1074D00000F03AF8E168094A0906090F515CC84012
:1074E0000749086007480068FFF7C0FBF8BD0000C7
:1074F000002002408813000000100240CAC60008A5
:107500005C01002054010020044805490068C96856
:10751000044A4905490F515CC84070475C0100208E
:1075200000100240E3C60008044805490068C96825
:10753000044A8904490F515CC84070475C0100202F
:1075400000100240E3C6000870B51A4AD3681A4911
:107550000C2018408D0004280CD04E00082810D0B4
:107560000C2810D050680004410F0120C003491CB2
:10757000884070BD1068C00601D5084670BD284619
:1075800070BD304670BD98020C4C000F205C1B0291
:107590009C0FD368641CDB0301D5314603E01268FD
:1075A000D20600D4294603F082F822460023FDF7D4
:1075B000B5FD70BD0010024000093D00DAC60008AC
:1075C000FEB505007ED0FE4CE7680C20E66807405B
:1075D0000120000406402878C00747D0082F05D0B6
:1075E0000C2F0AD101200004864206D120688003B6
:1075F0003CD568680028E5D038E0012069680004BF
:10760000814203D121680143216011E00523012259
:107610001B0492049942216802D111432160F1E7D1
:1076200081432160216801400091206890432060DF
:10763000686800280DD0FFF7F7FA009005E0FFF723
:10764000F3FA0099401A64287BD820688003F6D5A5
:107650000CE0FFF7E9FA009005E0FFF7E5FA009982
:10766000401A6428F0D820688003F6D42878800770
:1076700056D50923E868042F0DD00C2F01D1002E18
:1076800009D000283CD02168994301432160FFF7CD
:10769000CBFA064628E02168490701D5002891D099
:1076A00061681F22120291432A691202114361602C
:1076B0002168994301432160FFF746FFE16809060D
:1076C0000A0F00E08BE1BF49895CC840BE490860F1
:1076D000BE480068FFF7CAFA002873D120E0FFF720
:1076E000A3FA801B0228AFD820684007F7D560684E
:1076F0001F210902884329690902084360600FE0DD
:107700002068400840002060FFF78EFA064604E03B
:10771000FFF78AFA801B022896D820684007F7D422
:107720002878C00660D5002F0CD0A86900284AD060
:107730002068FF21013108432060FFF775FA0646F3
:107740002EE0C1E02068800502D5A8690028A6D0F7
:107750006068072149038843296A084360606068BC
:10776000297F0002000A090608436060286A410B6D
:107770000120C003491C8840E16809060A0F9149AD
:10778000895CC8409049086090480068FFF76EFA2D
:10779000002817D128E0FFF747FA801B0228A2D85B
:1077A00020688005F7D56068072149038843296A66
:1077B000084360606068297F0002000A09060843E8
:1077C000606011E0E2E02168FF2001308143216028
:1077D000FFF72AFA064604E0FFF726FA801B022884
:1077E00072D820688005F7D42878794E000724D510
:1077F00068690028306910D0012108433061FFF723
:1078000013FA009005E0FFF70FFA0099401A0228DA
:107810005AD830698007F6D50FE040084000306143
:10782000FFF702FA009005E0FFF7FEF90099401A11
:10783000022849D830698007F6D42878400766D5F1
:1078400000200290A06BC00006D4A06B01210907A4
:107850000843A063012002905E480168C90511D465
:107860000168821511430160FFF7DEF9009005E021
:10787000FFF7DAF90099401A642825D855480068BE
:10788000C005F5D5FF20AA680130824203D13169D5
:107890000143316111E001218902002A07D005234B
:1078A0001B029A4203D132690A433261EFE732691F
:1078B00082433261306988433061A868002810D063
:1078C000FFF7B2F9009008E05FE0FFF7ADF901467D
:1078D0000098091A4048814257D830698005F4D58C
:1078E0000DE0FFF7A1F9009006E0FFF79DF9009980
:1078F000411A3948814248D830698005F5D4029848
:10790000002804D0A06B012109078843A063686A9E
:10791000002866D00C2F3ED00126360602282068AB
:1079200005D0B0432060FFF77FF905462FE0B04354
:107930002060FFF779F9074604E0FFF775F9C01BEF
:10794000022822D820688001F7D4E96AA86AE26890
:107950000843296BFD231B049A4311430843E0604D
:10796000206830432060FFF75FF9054604E0FFF729
:107970005BF9401B022808D820688001F7D530E069
:10798000FFF752F9401B022801D90320FEBD2068F1
:107990008001F5D425E00128F8D0E0680121090430
:1079A000AA6A014091421AD10F218904EA6A014072
:1079B000914214D1032189050840296B88420DE0CA
:1079C00000100240CAC600085C01002054010020DB
:1079D00040100240007000408813000001D00120D8
:1079E000FEBD0020FEBDF8B504000ED0FF27606A82
:1079F0000537002500280AD02561656126464036F6
:107A0000A562707C002807D00AE00120F8BD6068FC
:107A1000B842F3D0E561F1E73574204600F03EF856
:107A2000022171742068026840239A430260212376
:107A3000A26860689B021A4038401043E3688A02DB
:107A40001340184323690B40217D1843C907C90F10
:107A50000843A169931019400843E169382319408C
:107A60000843216A802319400843A16A9300194002
:107A7000084321680860A0690421000C0840616A7D
:107A8000102319400843216848602068C169914368
:107A9000C1616565012070740020F8BD10B586B025
:107AA000044614216846FDF782FB1049206888428D
:107AB00019D10F48416B821411434163C16A0122FD
:107AC0001143C162C06A002110400590E02000907F
:107AD0000220019003200390029104910520694641
:107AE0000007FEF7D1FF06B010BD000000300140D6
:107AF00000100240094910B5401E884201D90120FA
:107B000010BD074C60610321081F02F00BFE00202E
:107B1000A06107202061002010BD0000FFFFFF00D2
:107B200000E000E0F0B502462032137E012B1ED0AB
:107B3000012515760223537606687468B3687027AA
:107B4000BC430F68274377600068AC07A04205D0AC
:107B5000084CA04202D0084CA04204D180244968BD
:107B6000A34319438160557600201076F0BD0220B2
:107B7000F0BD0000000801400014014070B5050090
:107B800005D02C462034607E002802D006E001207B
:107B900070BD00202076284600F010F802206076A4
:107BA000291D286801F0E6FF0120A077A076E07685
:107BB000207760776076002070BD000000680121AA
:107BC0008907884204D10348816B012211438163F4
:107BD0007047000000100240F8B505460446203505
:107BE000287E012817D001262E760220687622688A
:107BF00090687727FF23B8431B02984390600A6878
:107C0000502A31D00EDC202A4BD006DC002A48D086
:107C1000102A3AD145E00220F8BD302A41D0402A4E
:107C200033D136E0602A27D0702A12D00120000319
:107C3000121A2AD0824228D1CB684A688968206803
:107C400001F0D1FF20688168012292031143816015
:107C50001BE0CB684A688968206801F0C4FF21688E
:107C600088683843886010E0CA684968206802F074
:107C700034F85021206806E0CA684968206802F09C
:107C80003DF86021206801F0B9FF6E76002028766B
:107C9000F8BDCA684968206802F01FF840212068D2
:107CA000F1E711462068EEE710B586B004461421CE
:107CB0006846FDF77CFA012120688907884212D1C5
:107CC0000A49CA6A02200243CA62C96A0190014095
:107CD00005914102009100210291039104906946AF
:107CE0000348FEF7D1FE06B010BD000000100240B0
:107CF00000040050F8B5064604462036307E0D4696
:107D000001280BD0012008273076002A08D0042A49
:107D100016D0082A2AD00C2A4DD137E00220F8BD0F
:107D2000206801F073FF2068816939438161206810
:107D3000816904229143816120688169EA6812E0C7
:107D4000206801F07BFF206881690122D202114383
:107D5000816120688269012189028A4382612068E9
:107D60008169EA6812021143816124E0206801F010
:107D70007EFF2068C1693943C1612068C16904225E
:107D80009143C1612068C169EA6812E0206801F08E
:107D900089FF2068C1690122D2021143C1612068B4
:107DA000C269012189028A43C2612068C169EA6807
:107DB00012021143C16100203076F8BD70B5050094
:107DC00005D02C462034607E002802D006E0012039
:107DD00070BD00202076284600F00FF80220607663
:107DE000291D286801F0C6FE0120A077A076E07664
:107DF000207760776076002070BD704770B50546CB
:107E00002C4602202034002908D004290BD0082950
:107E10000ED0627F012A10D0012070BDA27E012AFF
:107E2000FAD1A0760AE0E27E012AF5D1E07605E0FB
:107E3000227F012AF0D1207700E0607701222868B4
:107E400001F0C4FE0122286892070121904205D06A
:107E5000074A904202D0074A904204D182685207F2
:107E6000520F062A02D002680A430260002070BD49
:107E7000000801400014014070B504460D4600683A
:107E8000002201F0A3FE2068016A0C4A114203D1CE
:107E9000016849084900016001202034002D06D006
:107EA000042D06D0082D06D06077002070BDA07686
:107EB000FBE7E076F9E72077F7E700001111000013
:107EC0007047704770470000F8B502680446D069F3
:107ED00011689668814B05461D402023002D6CD00B
:107EE000F7077F4DFF0FBC460D402F4379D0254645
:107EF000C7078035002F06D0CF0504D501271762AC
:107F00002A683A432A60820708D5F20706D0276814
:107F100002223A622A6804273A432A60420708D5B7
:107F2000F20706D02668042232622A68022632430B
:107F30002A6002070AD50A461A406646324305D02F
:107F40002668082232622E6816432E60020508D584
:107F50004A0106D501222668D20232622A681A43F3
:107F60002A602A68002A30D0800606D5880604D503
:107F7000616E002901D020468847286821688968F9
:107F8000490602D42821084225D0204602F0D5F81F
:107F900020688168490619D5826840218A43826039
:107FA000206F002812D04F498163206FFEF7D2FB6B
:107FB00000280AD0206F816B06E0850611D58D065A
:107FC0000FD5616E77E020468847F8BD2046FFF761
:107FD00079FFF8BD05E02046FFF774FF0020286018
:107FE000F7E7256E012D56D1C50654D5CD0652D5DD
:107FF000102616622068816825464906403500290A
:108000002ADA226F116849680904090CE1D02F8B24
:108010008F42DED9698311680968890617D401681F
:1080200032019143016020688168490849008160FC
:1080300020688168402291438160E36700202066C8
:1080400020680168B1430160206FFEF761FB288B57
:10805000698B401A81B21AE0298B6A8B891A6A8B64
:1080600089B2002AB5D00029B3D00268FF25213596
:10807000AA43026020688268520852008260E36767
:1080800000202066606620680268B24302602046D5
:10809000FFF716FF9DE7C50208D5750206D501203A
:1080A000000510622046FFF70CFF92E7050605D594
:1080B0000D0603D5A16E002985D18AE7400688D533
:1080C000480686D5116820464024A1431160836785
:1080D0000021816600F043F97BE700000F080000F3
:1080E0002001000461A0000810B5040003D0A06FB7
:1080F000002802D007E0012010BD002174200155A6
:10810000204600F027F82420A0672068016849086D
:1081100049000160204602F063F80128ECD0606A53
:10812000002802D0204601F07BFE20684168092229
:10813000D20291434160206881682A229143816084
:1081400020680168012211430160204601F0CEFE43
:1081500010BD0000F0B587B0064614216846FDF753
:1081600026F82C493068884251D12B48416B0122B6
:10817000920311434163C16A01221143C162C06A83
:1081800000251040059003204002009002200327A4
:1081900001A9A1C104200490052069460007FEF74B
:1081A00073FC1F4C1D48A560E56081C48027E56015
:1081B000A7602020256160610002A0611848083C8A
:1081C000FEF742FB002801D0FDF71EFE3467A662D1
:1081D000144C12482146143820600320606010209F
:1081E0000831A1C16561A561E56120462562FEF700
:1081F0002BFB002801D0FDF707FEF46600220121C9
:108200001B20A662FEF7A2FF1B20FEF793FF07B01C
:10821000F0BD000000380140001002403000024074
:108220006C160020B416002070B5C36F202B27D128
:1082300000290BD0002A09D0012483682403A3421B
:1082400006D10369002B03D1CB0701D0012070BDFB
:10825000034660331C7D012C12D001241C750023C1
:108260000366084C0368A34207D05C68240204D567
:108270001C680125AD062C431C6002F0B1F870BDEE
:10828000022070BD0048004070477047FFB50446AB
:10829000806F83B017460D4620285ED1002D0AD08E
:1082A000002F08D0A168C001814207D120690028B1
:1082B00004D1E80702D0012007B0F0BD20466030AD
:1082C0000090007D012848D0009801210175002010
:1082D000802108512120A067FEF7A6FC26464036E3
:1082E0000190378277820120A1680003814202D188
:1082F0002069002805D02F46002500990020087528
:1083000011E00027F9E700228021204602F0AEF8B4
:10831000002815D1002F15D02168387888627F1C7D
:10832000708A401E7082708A019B00280698009017
:10833000E9D100224021204602F098F8002808D018
:108340000320B9E728882168C005C00D8862AD1CEC
:10835000E6E72020A0670020AEE70220ACE77047E8
:10836000034D044C04A002F081F9E560FAE7000037
:108370000400FA0500ED00E0486172644661756C26
:10838000745F48616E646C65722E0D0A0000000017
:1083900030B585B014216846FCF709FF1148418BC0
:1083A000002901D10221418388B2012807D0022887
:1083B00003D100F003FCFDF749FC05B030BD0122FC
:1083C000094D940221462846FEF727FC0021012092
:1083D000029103910190009469462846FEF754FBF0
:1083E000EBE70000080100200004005010B5052450
:1083F0002407002204212046FEF70FFC002208215A
:108400002046FEF70AFC0A2002F095FB0122042117
:108410002046FEF702FC0A2002F08DFB0022042118
:108420002046FEF7FAFB10BD10B5052424070022F4
:1084300004212046FEF7F1FB012208212046FEF729
:10844000ECFB0A2002F077FB012204212046FEF714
:10845000E4FB0A2002F06FFB002204212046FEF715
:10846000DCFB10BDF8B50024052607462546360777
:10847000002204213046FEF7D0FB0A2002F05BFB0D
:10848000012204213046FEF7C8FB6006040E0821D5
:108490003046FEF7B5FB002801D0641CE4B205208D
:1084A00002F049FB6D1CEDB2082DE1D3002F03D083
:1084B000FFF79CFF2046F8BDFFF7B6FFFAE770B55F
:1084C000052605463607002204213046FEF7A5FBA7
:1084D0000024E80901D0012200E0002208213046F2
:1084E000FEF79BFB6806050E0A2002F024FB012222
:1084F00004213046FEF791FB0A2002F01CFB00220B
:1085000004213046FEF789FB0A2002F014FB641CAC
:10851000E4B2082CDDD370BD10B505242407012278
:1085200008212046FEF779FB012204212046FEF7B0
:1085300074FB002208212046FEF76FFB0A2002F0A0
:10854000FAFA002204212046FEF767FB10BD10B5A1
:1085500005242407002204212046FEF75EFB0022AA
:1085600008212046FEF759FB0A2002F0E4FA012216
:1085700004212046FEF751FB012208212046FEF788
:108580004CFB0A2002F0D7FA10BD70B505252D0767
:108590000024012208212846FEF73FFB062002F0B6
:1085A000CAFA012204212846FEF737FB062002F012
:1085B000C2FA07E0641CE4B2FA2C03D9FFF7C7FF44
:1085C000012070BD08212846FEF71AFB0028F1D1D2
:1085D000002204212846FEF720FB002070BD000089
:1085E000F8B501F0B5FC01F0EFFC58480068C0692F
:1085F000FDF7FAFC564C5749A082898F564E00254C
:10860000002931D0A26A730354499A4202DB022244
:108610000A7000E00D700A7801218902002A05D055
:10862000012A0ED0022A10D0032A1DD1608B012806
:108630002BD0022818D1454808214038FFF71CFCF0
:1086400012E0FF22F5329042F0D2608B01281AD05E
:10865000022804D008E03046FEF7DFFA04E03B4889
:1086600008214038FFF7CAFB0121C9023046FEF756
:10867000C7FA0127FF0300282AD039480560E079AE
:10868000002804D007E00022E5E70122E3E701200B
:10869000E07101F04DFF2078632806D900220821FF
:1086A0003046FEF7BAFA012205E0012208213046E1
:1086B000FEF7B3FA0022052039460007FEF7ADFAAF
:1086C000244C284E4034A08C274F012803D01CE0B6
:1086D000E5710022EAE725486946088072B68021E4
:1086E0002348FDF7A9FB002804D002226946204850
:1086F000FDF746FC62B61FA001F0B8FFA58403F0A9
:10870000F7FE642002F010FAFE60608C012808D1A8
:1087100010486584058003F0EBFE642002F004FA43
:10872000FE60208C012806D1258403F0E1FE642040
:1087300002F0FAF9FE600748124A0188914202D11C
:10874000C088002800D1FE60F8BD0000E8150020B8
:1087500008010020C00D002000040050810000200E
:108760004C0100200400FA0500ED00E0AAAA000078
:10877000384A0008BDF8C8EBC9FDBCB6C4A3CABDE1
:108780000D0A0000AA55000008B53721202000F08E
:108790006EF80321212000F06AF84021222000F029
:1087A00066F80821232000F062F8AA21302000F0AA
:1087B0005EF80A48008FC1B2322000F058F802215A
:1087C000332000F054F85F21202000F050F8684674
:1087D00000F006F80A2002F0AEF908BDC00D002036
:1087E00010B501460F2000F021F8002800D001202C
:1087F00010BD10B50446FFF78FFE3220FFF75FFE75
:10880000FFF7C3FEE0B2FFF75AFEFFF7BEFEFFF729
:1088100083FE3320FFF753FEFFF7B7FE0020FFF77C
:1088200021FE0446FFF793FE204610BD10B50C460E
:10883000FFF7DFFF2070012010BD70B50D46044624
:10884000FFF76AFE3220FFF73AFEFFF79EFEE0B226
:10885000FFF735FEFFF799FE2846FFF730FEFFF7DA
:1088600094FEFFF774FE0A2002F065F970BD10B5A2
:10887000FFF7E3FF012010BD10B50248FEF719FB1A
:1088800010BD000020150020FEB50446002772B67A
:10889000334A01688B1804D13248C768032080042A
:1088A000074088680190C868009048698E69002B6D
:1088B00008D12C4940398B6ACD042B438B628B6ADB
:1088C000AB438B62014631433CD025492368CB4200
:1088D00005D12449CA6803239B049A43CA602546EC
:1088E0002035002810D021680A6901231A430A6143
:1088F000216848610821204600F036F8032800D19D
:10890000A873216808204860002E10D020680169F3
:10891000012211430161206886611021204600F088
:1089200023F8032800D1A8732168102048600C4860
:108930002168C14206D10B48C168032292049143C9
:108940003943C16020680169490849000161216813
:108950000198886021680098C86062B6FEBD00007A
:108960000084FFBF4010024070B506460B480D461C
:10897000002409490068FCF7BBFB7D21C90048437E
:108980003168401E00D103240B682A469A4301D067
:108990000028F6D1204670BD204E00005C0100206A
:1089A0001CB5002116480091144A01910260C16370
:1089B0001205426081600722826301220261024641
:1089C000C16020321170FF235170C2334362816253
:1089D000117301638161042241634261C161FDF74A
:1089E000FDFC084800908013019069460448FDF79B
:1089F000A5FC00210248FDF74BFC1CBD00240140F2
:108A0000C41400200200000408B50848016B0122CC
:108A100011430163006B01211040009000220A20E5
:108A2000FEF794FB0A20FEF785FB08BD001002400C
:108A3000F0B587B014216846FCF7B9FB4748C26A15
:108A400004210A43C262C26A0A400592C16A8026B2
:108A50003143C162C16A31400591C16A0124214399
:108A6000C162C16A21400591C16A02252943C162E0
:108A7000C06A22462840059005201C210007FEF709
:108A8000CCF8012236493748FEF7C7F800223649AC
:108A90003448FEF7C2F891210520002209020007A0
:108AA000FEF7BBF831480190002705206946029780
:108AB00000940007FDF7E8FF0C20009011200190C2
:108AC000032003900520029769460007FDF7DCFFAD
:108AD00010206A46039591C2052069460007FDF7FC
:108AE000D3FF1120019002976946039700941D4817
:108AF000FDF7CAFF1E480190694600950294194887
:108B0000FDF7C2FFE0020090694601970295154803
:108B1000FDF7BAFF1748694691C1694611480397A6
:108B2000FDF7B2FF91200002694691C10520694618
:108B300000070397FDF7A8FF69460A4801970096CA
:108B40000294FDF7A1FF002201210520FEF7FEFAA5
:108B50000520FEF7EFFA07B0F0BD0000001002405C
:108B60000102000000040050083000000000111055
:108B7000000021100832000010B50F4C0D48206095
:108B8000FF20053060600020A060E060206160612F
:108B9000E0610121206249026062A161A0620720B8
:108BA000E0622046FEF71FFF206801684022114363
:108BB000016010BD003001405015002010B58AB092
:108BC00000240494059406940794089401211848FD
:108BD0000994009401940294890703940160092187
:108BE00084604160046113494461C160FEF7C6FFBF
:108BF00001200003049004A90D48FEF7EDFF0C4886
:108C0000FFF7DCF8089408A909480994FEF78AFFE1
:108C1000602000900848019002940822694603945D
:108C20000348FFF767F80248FFF73EF80AB010BDA7
:108C3000A8150020930400005702000000B585B07D
:108C400014216846FCF7B3FA0E480D490160E12192
:108C50004902416000218160C160016181610C2293
:108C6000C1614261016230214162012109038163D6
:108C70004900C163FFF738FA01F054FC05B000BDAC
:108C800000380140E815002070470000F0B589B0B9
:108C90000A2002F09BFC7D20C00002F0B1FCFF4CDA
:108CA0000025A570FE482065607B0C2801D30B20B1
:108CB0006073FC48E570FC4E00783071FB49A07988
:108CC000097840000843E17C89000843F071E06ABC
:108CD000F070010A3172401CE06260793146B07474
:108CE0004200B4310846A138FCF748FA6079F049EF
:108CF0008200400080191330121DFCF73FFA2A2031
:108D0000205E002803D0EB49098A08186085607945
:108D100006214843E44EE149821922310B7AD3758A
:108D2000497A117606217172E349DC4A0978B172F9
:108D3000217F317331461339937F0B75D27F4A758A
:108D4000002213311C3002F02BFD607906214843CC
:108D500000211C3002F036FD022002F087FCF57184
:108D6000E573A57201202073E572D448FEF77CF903
:108D700060840646E5706079FCF7E0FCD04AD14B90
:108D8000FCF7C0FB01F06CFE012300229B07FCF7FF
:108D900007FBFCF733FD0006C00C801980B20121EF
:108DA000C903A084884201D3401AA084C648E06366
:108DB0002079401C2071C148FEF756F92084BA483A
:108DC0000C300646423640300390C3E1BB48FEF704
:108DD0004BF92084BD4F0BE0B848FEF745F980B24F
:108DE0002084A18C884203D3B94A8918884206D3CB
:108DF00000210F2002F06AFB38422063ECD0206B88
:108E0000411C21D040047DD58122D20100210F20B8
:108E100002F09BFC7D20C00002F0F2FB002002F07B
:108E2000A4FB0021102002F051FB41069E48490E90
:108E3000274600225030E16402F07EFB9A48503011
:108E4000417A0729C1D101E001F08EFC0222A1493B
:108E5000401DFCF7B7F90028B7D102F004FDF96511
:108E6000B86502F0EDFC79663866F8786946401C12
:108E7000F8708D484D3002790A7040794870088842
:108E80000490F98B88427DD1934F308A38800399C2
:108E90008248898A41838948FEF7E6F8208402F0F7
:108EA00027FAFF22216E5204606E00238918584170
:108EB0000206080A1043410849000090080E090202
:108EC000A166E0667848E36D0A30A26D02F0A0FC6E
:108ED0006079636E81007448226E0818163002F0C3
:108EE00097FC7148E36E1230A26E02F091FC6E485E
:108EF00008214172A07C002816D06B4802227549D7
:108F0000553000E019E1FCF75DF900280CD1012093
:108F10006549E073C871E06C66311638C2B2084624
:108F20002274EA30FCF72AF96079002280005E4959
:108F30001C3002F035FC6079002180001C3002F00A
:108F400041FC009802F03BFB012002F08FFB2072F5
:108F500002216248FDF754FE00287DD000215348CD
:108F60004E4A0170B0891087F1895187A26B504B2E
:108F7000E2631A601A46C43AD27C13071B0F032B14
:108F800002D000E07AE063741209A2742571012313
:108F9000424AA3729087D187E372608B5049FF30B9
:108FA000C33080B2608388420BD949424018608345
:108FB00038887D21401C80B2C9003880884200D3A7
:108FC0003D803E887D20C000618B70434018206446
:108FD00007904448302107784348A77300884843E6
:108FE000FCF791FB01900A2031464143A08B3022CF
:108FF00005905043081AFCF77BFB0199FCF785F9B3
:109000007F21C905FCF7EBF8FCF7BFFB80B23549BF
:109010007F1E0880B84201D10120E072E68416204C
:10902000205EFCF777FB06900F46208CFCF786FB52
:109030002E4A2F4BFCF766FA064604910798FCF778
:1090400069FB3246049BFCF74FFA3B46069AFCF755
:10905000A7F9FCF7AFFB00E007E06064059800F0BB
:10906000C1FC207A002802D07DE0012177E70021B1
:109070000F2002F02BFA0006F9D574E0FCF79CFFF4
:109080000B4A0321303211540449B2890A87F2890C
:109090004A8707498000303942182BE070000020D1
:1090A0003F420F0008010020341200204801002038
:1090B00048130020000E0020180100202015002079
:1090C000B81E85EB51B8CE3FA086010000D0272402
:1090D000983A00002C0100204401002000040050B8
:1090E000E70300002401002028010020F853E3A535
:1090F0009B843E4003990190098B11804349BA6BD0
:1091000041184A6042497B6E401816303A6E02F0B0
:109110007FFB396DB86B884200DA38653B49019AAC
:1091200030398958814215DD002913D0002811DD1E
:109130000498F883022038700CE03A4600210F2092
:1091400002F003FB6079E178401C814202D00020EC
:1091500002F00BFA218CA08C814200D236E62D4A17
:1091600080188142FAD8A07A012801D00220A0728A
:1091700002F0BEF8284A00210F2002F0E6FA20791A
:10918000002806D025490A2209885143814200D28D
:109190002570E07B00281ED01C493C310B784878B4
:1091A0008A78022B17D110280CD0C82813D21C4B58
:1091B000C91C1818FBF7E2FF03F09AF9642001F0CC
:1091C000B3FC41E6174D28684000000E03D1C87873
:1091D000FCF799FA28600D4D0020603D2E4622785C
:1091E0006379183607E041006F5A715A8F4200D0F8
:1091F0000222401CC0B29842F5D32270064A0021D8
:1092000080320F2002F0A1FA09B0F0BD481300200F
:1092100034120020983A000000D0272418010020C2
:10922000C00D00203001002070470000F0B58DB067
:10923000002005900A2002F0C9F97D20C00002F04C
:10924000DFF9BD4800218170C26ABC4D521CC26268
:109250000175294613310A9112310991B849044622
:1092600022300891039028462F461338363707904E
:10927000613006900926B348667100782871B249BA
:10928000A079097840000843E17C12228900084354
:10929000E871A08DE870000A2872A849AE74B43154
:1092A0000A98FBF76BFF2822A8490998FBF766FF8D
:1092B0000898618D008A401860850398017AF975D5
:1092C000407A3876A2486E720078A872207F2873A0
:1092D000207D410098487C30091807980A7802756B
:1092E0004978417552200022944902F059FA607978
:1092F0000621484300211C3002F064FA022002F0EB
:10930000B5F9944E00210F2002F0E0F830422063BE
:10931000F8D0206B411C18D040047DD58122D201A9
:1093200000210F2002F011FA0021102002F0CEF8E7
:1093300041068248490E0022503002F0FDF87F4875
:109340005030417A022902D014E001F00DFA0222D5
:109350008149401DFBF736FF00280BD1207D0222FA
:10936000410075487C30091874485130FBF72AFFDA
:10937000002808D0217D79488A0074498C318850B2
:1093800001206070AEE002F06EFAE165A06502F0C7
:1093900057FA616620660598002844D1012005909F
:1093A00006986F4E008A3080644863494C30808A4A
:1093B00048836C48FDF758FE2084608B6A49FF3073
:1093C000C33080B2608388420CD949424018608320
:1093D00030886549401C80B20B313080884201D30F
:1093E0000020308030887D22D20001465143628BBC
:1093F000891821645D490E8801460A39F2B209B222
:10940000A2732185002903DA7D23DB00C918218599
:10941000521E964203D100E081E00121E172E08416
:10942000A08B00F0DFFA0698694682890A80C0891D
:1094300048804249042251310846A238FBF79EFE7B
:10944000207D00998200414800238C308150FF220A
:10945000216E5204606E8918584100060E0A0643B8
:10946000304602F0ACF870084000010E0002E166E0
:10947000A066324800264838E36DA26D02F0C8F9B4
:109480002E48636E4438226E02F0C2F92B48E36E18
:109490004038A26E02F0BCF92849002252393C2023
:1094A00002F07EF900213C2002F08CF9012002F04C
:1094B000DDF82072A0780121401CA0700520C903AE
:1094C0000007FCF78DFD207A002805D100210F2030
:1094D00001F0FCFF0006F9D5802200210F2002F0E8
:1094E00034F96670207D401CC0B220750A2800D275
:1094F000C0E60598002810D1A28B1D492046002AFD
:1095000002D00B889A4201D9098881831949A08B1E
:109510000988401E4843184908800DB0F0BD207DE1
:109520000E49820009488C308150144A00210F20D6
:1095300002F00BF924E70000700000203412002034
:10954000000E0020080100204801002048130020E0
:109550001801002000D027242C010020FFFF01006B
:109560004401002020150020E70300002401002012
:109570001401002012010020100100200090272477
:10958000F8B531492F48086002F056FA2F4800F02C
:10959000E9F92F4CE0822D48801C00F0E3F920838C
:1095A0002A48001D00F0DEF960832B4829494180DC
:1095B000014640310979294F0906090E617006D12B
:1095C000C7800121C1870A21418700218187244A60
:1095D000C18E1170C18F6171818FA171817AE1702B
:1095E0008588052165626181C6883046FBF780FD6C
:1095F000A08101462846FBF77BFD8800081885B24C
:10960000164825816843FCF799F8164A164BFBF774
:10961000E1FFFCF7F3F8E081658231463846FBF75D
:1096200067FD20820146C820FBF762FD20840120EF
:10963000A083FCF7D9FCA082E2890C490C48FDF715
:1096400017FDF8BD5DA5000868000020004F000868
:10965000080100201B020000C00D0020E8030000EC
:1096600018000020F853E3A59B843E40FF7F0000D4
:1096700020150020F0B5964D85B001202880954F2B
:10968000C820954C3880E079401CE071C00706D0B6
:10969000A08B411EA183022801D2C820A083A08BE9
:1096A00000F0A0F90A2001F091FF7D20C00001F038
:1096B000A7FF02218948FDF7A3FA002838D000202F
:1096C000874980000978884E490008438549097810
:1096D0000843B072102070728448C1887D20C00099
:1096E000FBF706FD7073824880490078B0733046FE
:1096F0000B308A780270C9784170411C7B48203059
:10970000027ECA70407E087178482230027E4A711B
:10971000407E887100220C39152002F041F80021AA
:10972000152002F04FF8022001F0A0FF714E03E077
:109730000120C5E7FEF754FF00210F2001F0C6FE0F
:1097400030422063F6D0206B411C7DD040047CD594
:109750008122D20100210F2001F0F7FF002110200B
:1097600001F0B4FE41066048490E00225030E16429
:1097700001F0E2FE5C4E5036707A112865D102226B
:109780005D49701DFBF71EFD00285ED1F01E0279B9
:1097900069460A7040794870B17A2980C820FBF781
:1097A000A7FC3880307BA083544DB01E008A2880EF
:1097B0004949301F808A48835148FDF755FC80B2E3
:1097C00020840390608B4F49FF30C33080B26083A8
:1097D00088420CD949424018608328884949401C76
:1097E00080B20B312880884201D3002028802D8848
:1097F0007D20C000618B684340182064019042487E
:10980000067828460A3800B2A6732085002803DAB5
:109810007D21C90040182085388830214843FBF756
:1098200072FF07462820205EFBF762FF3946FBF7F0
:109830006CFD7F21C905FBF7D2FCFBF7A6FF32497F
:1098400080B20880761E01E03FE03CE0B04201D1EA
:109850000120E072E5841620205EFBF75BFF02909A
:109860000F460398FBF76AFF284A294BFBF74AFE8D
:1098700005460E460198FBF74DFF2A463346FBF797
:1098800033FE3B46029AFBF78BFDFBF793FF6064C8
:1098900068460088E083144813495030807C633167
:1098A0006071420008460D465130FBF767FC607955
:1098B000294642000C48CC30FBF760FCA08BFF2807
:1098C00001D00320207005B0F0BD00F04DFF000076
:1098D0001801002028010020700000200004005022
:1098E0000D0100200E01002034120020C00D0020C8
:1098F0001800002000D027242C0100204401002063
:1099000020150020E703000024010020F853E3A500
:109910009B843E4070B586B014216846FBF747FC37
:1099200001250F4EED03002229463046FDF775F95B
:10993000012000240190029469460095039430466A
:10994000FDF7A2F803200190029469460095039464
:109950003046FDF799F8022001F0E6F806B070BD38
:10996000000400500088704770470000F8B50446B6
:1099700000206A461080194D55222A70AA226A706A
:109980000322AA70661DEE702A716971144A49009B
:109990008918AC712246E81DFBF7F0FB002007E0B8
:1099A00029186A468978128889186A461180401CED
:1099B000B042F5DB611DA81CFCF76CF90146684656
:1099C000018029190078C8716846407808722146DC
:1099D0000931024800F0D2FBF8BD000060140020FD
:1099E000C00D002010B51B4C228A01E0891AA1830A
:1099F000A18B9142FAD2228C8BB253431B18E38382
:109A0000132902D14A431018E083E08B30214843E8
:109A1000642164304843104960630968401A4B214F
:109A2000090140182063FBF775FE0C4A0C4BFBF74D
:109A3000D1FDFBF7BFFE0B49E062884202DD4A42DE
:109A40008018E062002801DA4018E06206490968DF
:109A5000486110BD08010020B4000020F853E3A5C0
:109A60009B843E40FF7F000020150020034A1168C0
:109A7000382389B299430143116070470030014097
:109A800010B5FDF7D7F810BD10B59AB0342168466F
:109A9000FBF78DFB14210DA8FBF789FB1C2112A8F5
:109AA000FBF785FB1B4801680324E402A143C214B1
:109AB00089180160FDF756FB17480169A143016150
:109AC00006200090FF20013002900120039010201A
:109AD00004900220099040040B90000100240C9097
:109AE0000A946846FDF76CFD0F200D9003200E9040
:109AF0000F941094012111940DA8FDF737FC8120DB
:109B00001290032080041890149412A8FDF77CFB97
:109B10001AB010BD007000404010024010480168AB
:109B2000821511430160C1680E4A1140C16001688D
:109B30000D4A11400160816849084900816001684F
:109B40000122920491430160C168FD2212049143F5
:109B5000C160002101610649044888607047000027
:109B6000001002400C40FF88F6FFF6FE005000088F
:109B700000ED00E070B5026801239B07114C124D07
:109B8000984203D0A04201D0A84203D17026B2432C
:109B90004E683243984203D0A04201D0A84204D17B
:109BA00003231B029A43CB681A4380239A430B6911
:109BB0001A4302608A68C2620968816201214161B8
:109BC00070BD0000000801400014014010B5CB0634
:109BD000DB0E0121046A99408C430462016A9A40B9
:109BE0001143016210BD30B58468FF252D021B02B0
:109BF0001343AC430B432343836030BD826870231F
:109C00009A430A4307210A438260704730B5026ACB
:109C1000520852000262026A456883697024A343B5
:109C20009C080B68A40023430224A2438C6845606F
:109C30001443836149684163046230BD30B5026AF0
:109C400010239A430262036A4568826973242402DE
:109C5000A2430C6824021443202293438A6845607F
:109C600012011A43846149688163026230BD30B5D4
:109C7000026AFF2301339A430262026A4568C3699C
:109C80007024A3439C080B68A400234301246402AE
:109C9000A2438C68456024021443C3614968C163D0
:109CA000046230BD30B5026A01231B039A4302628D
:109CB000036A4568C26973242402A2430C68240223
:109CC00014430122520393438A68456012031A43E6
:109CD000C46149680164026230BD30B5036A046A38
:109CE0006408640004628469F025AC4312012243D5
:109CF0000A24A3430B438261036230BD30B5036A7B
:109D00001024A34303628469036A0F252D03120301
:109D1000AC432243A024A343090119438261016299
:109D200030BD0000F8B5102605252D07AE62AF2026
:109D3000800000F000FFFCF7EBF930482E49006886
:109D4000FBF7A6FAFBF708FD2D4C6085AE6101F02C
:109D5000D1FB2C4F2C4E60650EE001F0CBFB606513
:109D6000FEF73EFC606B411C6163142804D927A0F8
:109D700000F07CFC2948C760606DB042EDD1002640
:109D8000666320780127FF03030000F0A8FC0504A8
:109D90000C192D303200012239462846FCF73DFFD0
:109DA000FFF768FC06E0012239462846FCF735FF3C
:109DB000FFF73CFA002239462846FCF72EFF18E050
:109DC000607A0122401E607239462846FCF725FF62
:109DD000FCF726F9002239462846FCF71EFF607A78
:109DE000002806D1267004E0FEF750FF01E0FFF7DF
:109DF0001DFA01F065FAF8BD0000C842000000201D
:109E0000700000200400FA053001CADE44572049E2
:109E100044204552524F522E0D0A000000ED00E042
:109E200010B5818CC90707D001684A6801235B041B
:109E30009A43836A1A434A60818C890707D501686F
:109E40004A6801231B049A43C36A1A434A60818CFF
:109E5000490707D501684A6801239B049A43036BAD
:109E60001A434A60818C090707D501684A680123B3
:109E7000DB039A43436B1A434A60818CC90607D5BA
:109E80000268916801231B039943836B1943916016
:109E9000818C890607D501688A6801235B039A4390
:109EA000C36B1A438A60818C490612D503685A68CD
:109EB00001210905046C8A4322435A60026C8A42DC
:109EC00007D10268516803235B059943436C19432A
:109ED0005160818C090607D501684A680123DB04BB
:109EE000806C9A4302434A6010BD0000F8B50446F6
:109EF000002680300660FCF797FE05462068006863
:109F0000124F000709D501212B46002249052046A2
:109F1000009700F0ABFA00280DD1206800684007D8
:109F20000BD501212B46002289052046009700F021
:109F30009DFA002801D00320F8BD2020A067E0672B
:109F40002666603426750020F8BD0000FFFFFF0183
:109F5000F8B5184CC826E078002829D16079002887
:109F600026D101206071144D686B002700281ED097
:109F7000686BC821081A15E01048E168405C616907
:109F800088470F480A21008848430E490880E06846
:109F9000401CE060E068C82800DBE760696BC8200F
:109FA000401A761EE168814201D0002EE4DC677120
:109FB000F8BD00005400002000000240F80C002012
:109FC000180100202A01002070B5224CE0780028FA
:109FD0003FD1207900283CD1012020711E4EF1692B
:109FE00000250906002933DA2156625791420AD129
:109FF000F06940062CD5A079002829D0A5712089C8
:10A00000401C208124E0A179002903D1A0710A20FD
:10A0100000F091FD00202056CC2148430F49421802
:10A02000206912181279B262401C00222061A256E7
:10A03000CC235A43895881420ADC25612078401C90
:10A04000207020780E2800D12570A078401CA070C8
:10A05000257170BD5400002000380140D00100205F
:10A0600010B5806A0022014640314A834A82FDF7DA
:10A0700029FF10BD70B5846AA06FE56F21688968FB
:10A0800000260906002906DA212804D152200653A9
:10A09000204600F06BF820688068400606D5222D27
:10A0A00004D15A200653204600F047F8204680305D
:10A0B00001681022114301602046FDF703FF70BDC7
:10A0C00010B501460968806A096889061CD4002217
:10A0D0005A210A5201680A68FF2301339A430A6031
:10A0E00001688A68520852008A6001688A684023C1
:10A0F0009A438A602021C167016E012904D1016859
:10A100000A6810239A430A60016E012902D0FEF703
:10A11000BBF810BD5821095AFDF7D2FE10BD10B58D
:10A12000806A016E012902D0FEF7AFF810BD5821F8
:10A13000095A4908FDF7C4FE10BD01680A68FF23EB
:10A1400021339A430A6001688A68520852008A6083
:10A15000016E012904D101680A6810239A430A603C
:10A160002021C167002101664166704701680A68C5
:10A17000C0239A430A6020218167704770B5164C4E
:10A18000E278002A0CD12279002A09D10122E2705A
:10A190000025C82903DC0222A256002A01DCE57052
:10A1A00070BD0123E356CC2253430C4AD150012306
:10A1B000E356CC2673439B180A460146181DFAF74E
:10A1C000DDFF6078401C607060780E2800D16570FB
:10A1D000A078401EA070E2E754000020D0010020CB
:10A1E000F8B50446016880682369E6691843636925
:10A1F000002533431843724A0B68724E33400343C1
:10A200000B602168486803231B039843E3681843E5
:10A2100048602168A069914201D0236A18438B6885
:10A220000B263602B34303438B60674923686748B4
:10A230008B420CD1C0688007800F06D0012839D02E
:10A24000022835D0032821D11EE001271FE06049F4
:10A250008B420AD1C0680C21084027D0042829D09D
:10A26000082825D00C2811D10EE093420ED1C168E8
:10A2700003208002014019D001208002091A19D060
:10A28000091A15D0814201D1082700E010274F4953
:10A29000504840398600934232D1002F0CD0022F13
:10A2A0000DD0042F10D0082F7FD126E00027EEE735
:10A2B0000227ECE70427EAE7FDF726F906E009683C
:10A2C000C90605D4304603E0FDF73EF9002872D0F8
:10A2D000626851005118814267D81103814264D3EA
:10A2E000010E06025008002330185941FAF716FFF4
:10A2F00003210902411A384A55E00120C003E7E76B
:10A300000122E369D20393422BD13B0000F0E7F92D
:10A310000906090C4D114D4D4D274D00FDF7F4F880
:10A3200009E0FDF701F906E00968C90605D43046E1
:10A3300003E0FDF709F900283DD0616840004A08B4
:10A340008018FAF7D5FE80B20146244A10399142AE
:10A350002BD8511C01400007400F084329E010464C
:10A36000EBE73B0000F0BBF90906090C21122121A3
:10A3700021232100FDF7C8F80AE0FDF7D5F807E032
:10A380000968C90606D4304604E00EE0FDF7DCF8A3
:10A39000002810D061684A081018FAF7A9FE80B2A8
:10A3A00001460E4A1039914203D9012503E01046B7
:10A3B000F0E72168C86000206066A0662846F8BD06
:10A3C00000480040F369FFEF0038014040100240B0
:10A3D0000044004000093D00FFFC0F00EFFF0000BB
:10A3E000F8B5044641654030002627460283803791
:10A3F0003E602220E0672546206F603500281CD093
:10A400001749C162216F17480863216F16484863D6
:10A41000206F8663236F606D9C4613462168024659
:10A4200060462431FCF758FA002806D01020386026
:10A430002E752020A0670120F8BD2E7520680168C8
:10A44000FF2201321143016020688168012211431B
:10A450008160206881684022114381600020F8BD3E
:10A46000C1A000081FA1000875A00008FFB581B0B9
:10A4700005460F46044660350A9E39E0701C37D009
:10A48000FCF7D2FB0499401AB04222D8002E20D00B
:10A490002068016849072BD5C069C043000527D44F
:10A4A00001202168C002086220680168FF22A132F1
:10A4B000914301602068816849084900816020203B
:10A4C000A067E0678034206000202875032005B075
:10A4D000F0BD20680168FF22A1329143016020682D
:10A4E00081684908490081602020A067E067EBE7A8
:10A4F0002068C1693846884305D00021039881420D
:10A50000BCD00020E3E70121F8E7000010B50449C2
:10A510001020096808620248FDF7D6FC10BD000053
:10A52000E815002001490D20887070475400002074
:10A5300010B507480A22018A51434184FEF764FAA4
:10A54000FEF77CFBC82203490348FDF76DFE10BDF2
:10A5500008010020F80C0020E8150020F8B53E4C5A
:10A56000002321783D4A1D46082910D0072947D0ED
:10A57000062950D0052952D0042953D0032954D09C
:10A58000002956D0012958D002295AD05BE0A17881
:10A5900000264A1F04E0314FBF5DFB189BB2761CBA
:10A5A0009642F8DB667927799A195118E378627830
:10A5B000C9188918C9194018C0430006000E1AD1DD
:10A5C000012E14D0022E16D125482449C018FAF7BE
:10A5D000D5FD01F08DFF642000F0A6FABFF34F8F88
:10A5E00021492048C860BFF34F8F00BFFDE75908DD
:10A5F0001046FFF7BBF92570E570A570A571F8BD91
:10A60000A1795054491CC8B2A071A178491F884251
:10A61000F5D1082001E0607007202070F8BDE070DF
:10A620000620FAE760710520F7E7A070E5700420C6
:10A63000F3E7552807D10120EFE7AA2803D102202C
:10A64000EBE7032803D02570E570A570F8BD032063
:10A6500020702071F8BD000000010020FC130020D4
:10A66000C00D00200400FA0500ED00E010B5024A1C
:10A67000024900F0E5F910BD29B80008600100208A
:10A680002021020C01D010211046020A01D01046F0
:10A690000839020901D01046091F820801D010466E
:10A6A000891E420801D0881E7047081A7047F8B505
:10A6B000040C8BB2264682B25E430D0C1046370C5A
:10A6C0005843360480190021794116466E43370CF1
:10A6D00036048019794126466E438919F8BD30B495
:10A6E0007446641E2578641CAB4200D21D46635D2F
:10A6F0005B00E31830BC18474900CA02024310004F
:10A7000000D004204A0D01D001221043044A490D13
:10A71000914201D102210843012800D10520704750
:10A72000FF0700008307FF22DB0E9A408907090E0E
:10A730009940002808DB830809489B001B1818680B
:10A7400090430843186070470007000F08388308DB
:10A7500004489B001B18D86990430843D861704790
:10A7600000E400E000ED00E0BFF34F8F0449034830
:10A77000C860BFF34F8F00BFFDE700000400FA057B
:10A7800000ED00E0F8B504464F1EC8000838211857
:10A7900015461E46086849683A4606239A4310D073
:10A7A0002A463346FAF7AEFE3A46D200083AA318D4
:10A7B0001A687F1E5B68FAF7F3FD06223B46934357
:10A7C000EED1022F23D0042F11D0062F2FD12A46ED
:10A7D0003346FAF797FEE36AA26AFAF7E1FD2A46E2
:10A7E0003346FAF78FFE636A226AFAF7D9FD2A46E2
:10A7F0003346FAF787FEE369A269FAF7D1FD2A46E4
:10A800003346FAF77FFE63692269FAF7C9FD2A46E3
:10A810003346FAF777FEE368A268FAF7C1FD2A46E5
:10A820003346FAF76FFE63682268FAF7B9FDF8BDA0
:10A83000002210B5134610460149FAF7CBFE10BDB1
:10A840000000F03F10B5FAF7ABFD10BD002210B5C7
:10A85000134610461146FAF7BDFE10BD10B507218C
:10A86000024A00200907FAF72DFF10BD010300007E
:10A87000034A10B500201107FAF724FF10BD0000AD
:10A8800001FDFFFF02E008C8121F08C1002AFAD12B
:10A8900070477047002001E001C1121F002AFBD160
:10A8A0007047000001490860704700006401002003
:10A8B00008B50021684601706B46012202212C2058
:10A8C00000F052FF0221684601706B4601222C20E5
:10A8D00000F04AFF08BD000038B504466D20694607
:10A8E00008706B46012207492E2000F03DFF064903
:10A8F000002C01D0054A00E0054A2E2000F01AFF86
:10A9000038BD000006080000061800000706000019
:10A910000716000038B504466B4602220021362097
:10A9200000F0EEFDB3212300FFF7D9FE0E0F08154E
:10A930003A3A3A3A1C273A3A2F34483A00216846C4
:10A94000017040784108490014E0694608788008A1
:10A950008000401C04E06946087880088000801C64
:10A9600008701DE0684602780A404832027041785B
:10A97000802001436846417012E0684602780A4030
:10A98000027040784106490EF4E769464878022192
:10A99000084303E069464878FD210840694648704D
:10A9A0006B4601220021362000F0DEFE012200ABC2
:10A9B00011463620013300F0D7FE38BD69460878CD
:10A9C000CF21084069462030CAE708B50321684610
:10A9D0004170012101706B4602220021362000F0F7
:10A9E000C3FE0122D20306212D2000F0A3FE012088
:10A9F00000F09AF80120FFF78DFF08BD08B5020AA4
:10AA000069464A7008706B46022204212D2000F02E
:10AA1000ABFE0320694608706B46012206212D20FB
:10AA200000F0A2FE0020694608706B460122062154
:10AA30002D2000F099FE0A212D2000F047FD08BDD1
:10AA4000F8B516460F460446002503E03946B047E0
:10AA5000641C6D1C20780028F8D12846F8BD000041
:10AA6000F8B54A002B4B520DD6182B4A0C4605461A
:10AA7000142E2BDA002E12DA284BFAF791FC002262
:10AA80001346FAF701FF40D2002C03DA0124E40751
:10AA900000253AE02046284337D0214C14E0214FCE
:10AAA0000B46F7403B402B4331D01C4BFAF778FC68
:10AAB00000221346FAF7E8FE27D2002C03DD01201E
:10AAC0000005F0400419BC4300251EE0332E1EDCB7
:10AAD00033460027143BFF43DF40384217D00F4B6B
:10AAE000FAF708FD00221346FAF7CEFE0DD2002C2D
:10AAF0000ADD142E0CD03420811B0120884040191F
:10AB0000A84200D2641C0546BD4321462846F8BD34
:10AB1000641CF9E701FCFFFF9C7500883CE4377E6C
:10AB20000000F03FFFFF0F007D2110B5C900484332
:10AB300000F001F810BD002140E000BF00BF00BFE1
:10AB400000BF00BF00BF00BF00BF00BF00BF00BF0D
:10AB500000BF00BF00BF00BF00BF00BF00BF00BFFD
:10AB600000BF00BF00BF00BF00BF00BF00BF00BFED
:10AB700000BF00BF00BF00BF00BF00BF00BF00BFDD
:10AB800000BF00BF00BF00BF00BF00BF00BF00BFCD
:10AB900000BF00BF00BF00BF00BF00BF00BF00BFBD
:10ABA00000BF00BF00BF00BF00BF00BF00BF00BFAD
:10ABB00000BF00BF00BF00BF00BF491C8142BCD323
:10ABC0007047FFB581B01E460F46040026D00B9992
:10ABD00003980143A06A3943826807209047002800
:10ABE00018DB0A99A06A3143826806209047002842
:10ABF00010DB25462035A979032F01D90820014310
:10AC0000032E01D904200143A06A826809209047DD
:10AC1000002806DA0120C04305B0F0BD0020C04383
:10AC2000FAE7384600F000F92060304600F0FCF802
:10AC300060600A9868700398A870EF702E710B9886
:10AC400068710020E8E70000F7B50446002090B0E6
:10AC500000900190002C05D06A46062101F082FC8C
:10AC6000062803DA0020C04313B0F0BD68464078E0
:10AC700001026846007800040918684680780818C0
:10AC8000FAF75CFD054668460391007901026846C3
:10AC9000C07800040918684640790818FAF74EFD94
:10ACA000032206460F4692075C4BFAF7EDFD07D2EA
:10ACB00000225B4B30463946FAF716FC06460F4633
:10ACC00003229207554B28460399FAF7DDFD07D278
:10ACD0000022534B28460399FAF706FC05460391D8
:10ACE0002068FAF72BFD02460B4630463946FAF744
:10ACF00071FC07460A200791205EFAF70BFD3A46E1
:10AD0000079BFAF7FFFB064608200991205EFAF739
:10AD1000EFFC0021C943FAF736FBFAF78DFD324606
:10AD2000099BFAF73DFB069108906068FAF706FD6B
:10AD300002460B4628460399FAF74CFC05461A20B2
:10AD40000E46205EFAF7E6FC2A463346FAF7DAFBAF
:10AD50000C9009911620205EFAF7DCFC099B0C9AF6
:10AD6000FAF71EFB05910A902A46334638460799A2
:10AD7000FAF7C8FB059B0A9AFAF7C4FB05910A90FB
:10AD80001420205EFAF7C6FC3A46079BFAF7BAFB96
:10AD900007461C200791205EFAF7BCFC2A46334682
:10ADA000FAF7B0FB0E900B911820205EFAF7B2FC78
:10ADB0000B9B0E9AFAF7F4FA2A463346FAF7A2FBEF
:10ADC0000B910E902069FAF7A5FC0B9B0E9AFAF7EF
:10ADD000E7FA2A463346FAF795FB05460E46E06841
:10ADE000FAF798FC2A463346FAF7DAFA3A46079B0E
:10ADF000FAF7D6FA059B0A9AFAF7D2FA01229207D5
:10AE0000084BFAF77FFB02460B46129C08980699FE
:10AE100003C411980CC0002026E70000FFFF5F412B
:10AE200000007041E17A843F00B50121C9040300AC
:10AE3000FFF755FC081A05080B0E1114171A03200A
:10AE4000C00400BD0720C00400BD0F20C00400BD29
:10AE50001F20400300BD3F20400300BD7F20400372
:10AE600000BDFF20400300BD084600BDFEB5264FD3
:10AE70000D4604000FD0002D0DD0264600202036B0
:10AE8000B071F07129680D208847002801DA780038
:10AE9000FEBD102801D03846FEBDA562E968002934
:10AEA00001D028208847204600F030F80028F3DB46
:10AEB000A06AA52182680E209047A06A9621826828
:10AEC0000F209047A06A0221826862209047A06A02
:10AED000002182680E209047A06A002182680F201E
:10AEE00090477179302001910090062320220121A2
:10AEF0002046FFF766FE0028CEDB204600F0AEF8C5
:10AF00000028C9DB0020FEBDFFFFFFFF10B586B0A3
:10AF1000044614216846FAF74AF9002C7ED0A06A4C
:10AF2000122143686A4610209847122877D1684654
:10AF300000780122010168464078120300090818D0
:10AF400043492081884201DD801A20816846837848
:10AF500040780007000D18186081884201DD801AD2
:10AF6000608168460079012201016846C0781205B7
:10AF70000003091868464079000908183549E0605F
:10AF8000884201DD801AE060684640790007030BC3
:10AF90006846807900021B186846C079181820613D
:10AFA000884201DD801A20616846417A007A0002F9
:10AFB000081802B2284801210904A282824201DD58
:10AFC000521AA2826A46D37A927A12029A1812B25E
:10AFD000E282824201DD521AE2826A46537B127B90
:10AFE00012029A1812B22283824201DD521A22837F
:10AFF0006A46D37B927B12029A1812B26283824213
:10B0000001DD521A62836A46537C127C12029A183E
:10B0100012B2A283824204DD501A01E00BE008E084
:10B02000A083A06A016828208847002806DA01204A
:10B03000C04306B010BD0020C043FAE7C011C007EE
:10B040002034002800D0802060710020F1E700004B
:10B05000FF070000FFFF0700FF7F000010B504009E
:10B0600009D0A06A0721826808209047002805DAE5
:10B070000120C04310BD0020C04310BD0720203474
:10B080002070002010BD0000FEB504460020019095
:10B0900000906079734940000E5A61782578491E06
:10B0A0007148CFB20163042D77D0072D75D00021F0
:10B0B0000291217801736C49E37901229205896933
:10B0C000002B6CD0914381616748217A4173217ACA
:10B0D00082698907890B0A4382610021042000F0FC
:10B0E00034FB324661492E2000F024FB3846FFF73E
:10B0F000F3FB5F4E0522705D810040185D494318E7
:10B1000007212B2000F030FB5B49029801220B182D
:10B110000B21282000F028FB705D584980000A5858
:10B120000C21282000F011FBE079554980004018DF
:10B13000A1794900425A0221272000F0FBFA514828
:10B140007E00825B0421272000F0F4FAE0790028D9
:10B1500029D0A07804282CD0282069460872202203
:10B160000621272000F0E6FA02AB01222621272043
:10B1700000F0FAFA444938014018E1788900425851
:10B180000821272000F0E1FAA17A601C627A090206
:10B19000114313D016E000E001E0012188E71143DC
:10B1A000F608816190E764220621272000F0C2FAA8
:10B1B000E0E71020694608720246D1E73349017280
:10B1C000090A4172417A007A0A02024320212720AB
:10B1D00000F0B0FA2E4F0C2123203A6800F0B5FAA7
:10B1E000F01982880421232000F0A4FAA079002815
:10B1F0000BD0E0792749012243180021212000F0DB
:10B20000B3FA03200190012000902A07120F1001C9
:10B210000243607800218007000B0243019800057B
:10B2200002430098400402432079C00640090243CB
:10B230006079C00602431F2000F087FAA078617889
:10B240000123084302040848DB030261E179490352
:10B2500019430A4302610021082000F076FA002019
:10B26000FEBD000098C600089401002004280000DC
:10B2700040C60008240000204200002048C6000804
:10B2800068C6000874C6000878C6000841100000AF
:10B2900060C600084400002038B50C4607498A8B78
:10B2A000002102432C2000F045FA684604706B46EA
:10B2B000012206212C2000F057FA38BD940100200D
:10B2C00010B5FFF7F5FA10BD10B50446042136207D
:10B2D00000F0FCF80121C902002C01D0084300E075
:10B2E000884302460421362000F02FFA10BD0000EA
:10B2F00038B540206946087000210E2000F0E6F8BD
:10B300000446002211460E2000F01FFA6B4601226F
:10B3100000210D2000F028FA074A00210F2000F03C
:10B3200014FA00F0EDF9224600210E2000F00DFA8B
:10B3300002480021017338BDF8FF2724B401002022
:10B34000FEB50546042069460870514C0020607522
:10B3500021462031206348710873A0836063A06395
:10B3600000F0C8F84B4E206002E000F0C3F8206007
:10B37000B042FAD10020FFF7CDFA00F0BBF8464EFC
:10B3800020603078242801D9243806E00621F9F716
:10B39000AFFE0622101A40010843020601040A43C8
:10B3A00001020A430243B260706000211E2000F0D7
:10B3B000CCF900F09FF820606B4601220021242088
:10B3C00000F0D2F91E20FFF719FB86B2300AA073F5
:10B3D0000420FFF713FB074600F08CF820603806C6
:10B3E000000E0DD002206946087101AB0122122126
:10B3F0002D2000F0B9F9A08B012109030843A08397
:10B4000000F078F820600620FFF7F8FA6060072067
:10B41000FFF7F4FAA060F006C00E207501D11020ED
:10B420002075C0B200F0DCF9E80707D0FFF7CDFACD
:10B43000A08B0121C9020843A0830AE00521362020
:10B4400000F02EF81549084002460521362000F08C
:10B4500071F90120FFF75EFA0021042000F036F8B0
:10B46000A0610021262000F031F81521890308434E
:10B4700002460021262000F068F90022262136200D
:10B4800000F058F900F036F820600020FEBD000002
:10B49000940100203001CADE18000020FFFD0000EA
:10B4A00038B5094C89B280B26B46022200F028F808
:10B4B000002806D1684640780102684600780818DE
:10B4C00084B2204638BD0000FFFF000038B50024DC
:10B4D000E44389B280B26B46042200F011F80028E0
:10B4E00006D103216846435C2202D418491EFAD5CE
:10B4F000204638BD10B500210846FFF7E7FF10BD14
:10B5000038B5002909D0402420436C462070C8B2C9
:10B510007F2906D8607002200AE069460870012081
:10B5200006E0802420436C466070C809A0700320A8
:10B53000694600F0B7FF38BD10B5144603460A4609
:10B5400021461120FFF7DCFF10BD10B50346052290
:10B5500000211520FFF7D4FF10BD10B503460522CA
:10B5600000211720FFF7CCFF10BD38B5054600209D
:10B570006946087000F0C4F8FF2401342246002D0B
:10B5800001D00322120200210D2000F0D3F8002D7B
:10B5900013D06B46012203210F20FFF7B1FF68464D
:10B5A0000078000709D5FFF7A3FE224600210D20F1
:10B5B00000F0C0F80020C04338BD002038BD10B5F1
:10B5C000024601210A2000F0C0F810BD10B5044663
:10B5D00000211A20FFF77AFF000D22030005120B4D
:10B5E000024300211A2000F0B0F810BD10B5024649
:10B5F00002492E2000F09EF810BD00000418000043
:10B60000F8B505466B46012203210420FFF778FFB9
:10B610000126114C3607002D0DD02A4600210C20A2
:10B6200000F088F8694608781021084369460870D8
:10B63000A069304307E069460878EF210840694671
:10B640000870A069B0430B46A061012203210420C9
:10B6500000F08AF8F8BD00009401002010B5024601
:10B660000021182000F066F810BD0000F8B507466C
:10B67000002568460570B807204C2E4600280ADAD7
:10B680008020694608706B46012200210D2000F0E1
:10B690006BF801202073F8076946087821D006214D
:10B6A0000843694608706B46012200210D2000F016
:10B6B0005BF803210F20FFF7F3FE8121C900084248
:10B6C00019D04020694608706B46012200210D20E8
:10B6D00000F04AF80020FFF7F7FD00252673ED4340
:10B6E00009E002210843694608706B4601220021E7
:10B6F0000D2000F039F82846F8BD0000B401002004
:10B700001CB56B46012203210F20FFF7F9FE6846A6
:10B7100000784022C1091040C9014000814208D090
:10B72000012069460871024601AB03210D2000F09B
:10B730001BF81CBD08B56B461A70120A5A7089B204
:10B7400080B2022200F010F808BD38B500236C4624
:10B75000E254120A5B1C042BFADB89B280B2234646
:10B76000042200F001F838BD38B58024002909D042
:10B77000C02528436D462870C8B27F2907D8687055
:10B78000022009E0204369460870012004E02043BC
:10B790006870C809A8700320694600F02DFF38BD05
:10B7A00010B51446012312189B029A4202D90020B8
:10B7B000C04310BD0B46821E21460920FFF7D4FF6F
:10B7C000002010BD10B5054A8905126901430A43DE
:10B7D00000210820FFF7B9FF002010BD94010020D0
:10B7E00038B504466B4601220E212B20FFF788FE58
:10B7F00068460078E10640094001C90E01436846E9
:10B8000001706B4601220E212B20FFF7ADFF38BDE2
:10B8100010B5002142541C06120A22431B0A491C7F
:10B820000429F7DB10BD000013B501231A46694651
:10B830000248FCF72BFD00981CBD0000E815002015
:10B840007CB5002425466846FFF77FFE0420694644
:10B85000220E2D02154322020C5C1443401EF7D524
:10B86000204629467CBD7CB5002425466846FFF766
:10B8700074FE04206946220E2D02154322020C5C40
:10B880001443401EF7D5204629467CBDFBF7DAF964
:10B89000FEF7FAF8FDF7CCF841494248002522C0EE
:10B8A00005608561C56140490562C1600838FBF7E4
:10B8B00065FBFDF7A9F8FDF7C1F9FDF75DF9FDF7A7
:10B8C0006FF8052601223607D1033046FBF7A5F9AC
:10B8D000FDF756FEFCF758FFFAF73CFAFAF70AFABA
:10B8E000FCF756FD0721B015FFF7D6FCFFF7E8FC83
:10B8F0002E4C0A21208A01224843608411033046DD
:10B90000FBF78BF92748C8222949C830FCF78CFC83
:10B91000284F294E207900283FD0607800283CD05D
:10B92000FEF7B2F82571FAF73FFC20700F280AD90C
:10B93000012211033046FBF770F9FEF7F3F90022FC
:10B940000121090309E0012251033046FBF765F9A3
:10B95000FEF7E8F90022012149033046FBF75DF9C3
:10B96000FCF73EFE608C002801D0401E6084134826
:10B97000618C00780843CDD13878002801D00328A5
:10B98000C8D10121C9023046FBF73AF90028C1D1DC
:10B9900001210846FBF706FCBCE7FCF721FEB9E7EE
:10B9A000007C004020150020FFFF0000080100205F
:10B9B000F80C002081000020000400505A000020F4
:10B9C00010B586B01748FBF75CFA14216846F9F702
:10B9D000EEFB154800900320019000200290052006
:10B9E00069460007FBF750F869461048FBF74CF82A
:10B9F00069460F48FBF748F801210846FBF7D2FBE0
:10BA0000FF2401342046FBF7A5FB0A4908680422FD
:10BA1000104308602046FBF7ADFBFBF7B3FB06B015
:10BA200010BD000020150020FFFF000000040050A2
:10BA3000000800500070004010B501229202174922
:10BA40001748FAF713FA1548164902888A4224D093
:10BA50000180FF2101318180FF21F531C1800A2160
:10BA6000018100211E224181D24382810122C281B3
:10BA700081831E23C386022303877823438782871B
:10BA8000C28702464032118451849184C1839180DF
:10BA900014238382118200F02BFD10BDC00D002005
:10BAA00000FC0008AA550000F0B51FB496B084460B
:10BAB0000C460246199D18980390490068006300DF
:10BAC000490840080193002A01D0012600E0002621
:10BAD0009E19FE4BF6185B109E422BD36E00039FFF
:10BAE0000296002F00D00127F719F84EF84BBE1927
:10BAF0009E421FD3039E0346F64F334309D03B4675
:10BB00009C4201D1002A04D0019B002A05D00126C5
:10BB100004E0002039461BB0F0BD00269E19EE4B14
:10BB20009E4207D8039F029E002F00D00127F619DE
:10BB30009E4207D92B4660462146189AFEF782FEA0
:10BB40001BB0F0BD0023002C29DAE44EB04226DA07
:10BB5000E34EB04201DB022321E0DE4EB0421EDBA9
:10BB6000E04E070DBE19142E09DD3427BF1B039EBE
:10BB7000FE400196BE40039FBE420BD00FE0039FE4
:10BB8000002F0CD11427BF1B0646FE400196BE4075
:10BB9000864204D1019BDE07F60F02239B1B0E4653
:10BBA000164318D1002D16DA002C03D0022B01D039
:10BBB000012B06D00220FEF775FEFEF739FE1BB002
:10BBC000F0BD0220FEF76EFEFEF732FE0122D20724
:10BBD00051401BB0F0BD039E002E61D1BF4EB0425C
:10BBE00020D1C148844201D1002A08D0B9488142FD
:10BBF00009DB002D10DB189829461BB0F0BD002092
:10BC0000B4491BB0F0BD002D06DA01222946D20747
:10BC1000189851401BB0F0BDB44979440868496890
:10BC20001BB0F0BDAB4FB84225D1002D1FDA002963
:10BC300004D0B14212D1002A09D018E0002A72D1F2
:10BC4000A649E20F0020D20711431BB0F0BD00202F
:10BC5000E20F0146D20711431BB0F0BDB14206DA34
:10BC6000234600203946F9F7B5FC1BB0F0BD10465D
:10BC700021461BB0F0BDB14212DA0126B607B5422B
:10BC800003D1234610461946FEE3994EB54207D12B
:10BC9000261E05DB1046314600F040FC1BB0F0BD0F
:10BCA00067007F081646002A40D100290AD08B4A37
:10BCB000914229D1002C0EDD002D1CDB0020114605
:10BCC0001BB0F0BD022B16D0002C14D0012B12D1CA
:10BCD000002C14DB0FE0002C28DA002D09DB012BEF
:10BCE00003D000207D491BB0F0BD002081491BB06E
:10BCF000F0BD012B03D0002001461BB0F0BD002099
:10BD00000121C9071BB0F0BD724A91420ED1002C2F
:10BD100001DA002B17D0022B06D00020C043F9F720
:10BD2000F9FC1BB0F0BD90E20120F8E7E217521CCD
:10BD300094461A4307D000220892664C62465B1E66
:10BD40001A4307D009E00120FEF7ACFDFEF77EFDA7
:10BD50001BB0F0BD0022644C0892674A90427DDD22
:10BD6000664B674A98421FDD914202DC002D05DBDD
:10BD70004DE05848814217DB002D48DD0220FEF7D8
:10BD800091FDFEF76BFD05460E460022534B214602
:10BD90000898F9F7B7FB084671004908C00FC007BB
:10BDA000014328461BB0F0BD914215DA002D2EDA72
:10BDB0000220FEF777FDFEF751FD05460E460022F4
:10BDC000464B21460898F9F79DFB72005208C80FB0
:10BDD000C0070243114617E03E4B994223DD002D78
:10BDE00015DD0220FEF75EFDFEF738FD05460E4626
:10BDF00000223A4B21460898F9F784FB0846710067
:10BE00004908C00FC007014328461BB0F0BD0220FF
:10BE1000FEF748FDFEF72CFD49004908E20FD20766
:10BE200011431BB0F0BD002230463946F9F75CFBE8
:10BE3000012205460E46D243F9F744FC314A324B03
:10BE4000F9F758FB2A463346F9F75CFB0022284BEA
:10BE5000F9F750FB07462A46334600E064E00391B9
:10BE600010461946F9F74EFB3A46039BF9F74AFB91
:10BE70000746032209915207244B28463146F9F719
:10BE800041FB07910C90224A204B38460999F9F75B
:10BE900039FB074601911F4A1F4B28463146F9F7E7
:10BEA00031FB3A46019BF9F71FFB07460B4602465A
:10BEB000099107990C98F9F773FA00250E46284660
:10BEC000079B0C9AF9F710FB3A4627E0FFFF1F008B
:10BED000FFFF0F000000F03F0000E0FF0000F07FD8
:10BEE0000000404301FCFFFF0000F0BF5A0B0000C0
:10BEF0000000E03F0000F0FF0000E0410000F043E0
:10BF0000FFFFEF3F555555555555D53F4715F73F61
:10BF1000FE822B6544DF5DF80BAE543E099BF9F7BA
:10BF2000E9FA02460B4652E1012500202D05A942FF
:10BF300007DA352230463946F9F7C4FB0646342085
:10BF4000C0430A151218FE48101803900803FD4953
:10BF5000000B01430F46FC49884201DC002003E04E
:10BF6000FA49884202DA0120119005E00020119080
:10BF70000398401C7F1B039011980597C200F4485A
:10BF80000F927844801843680268394630460D9312
:10BF90000292F9F7A9FA07910C9030460D9B029A8C
:10BFA0000599F9F7FDF902460B460020E549F9F736
:10BFB00011FB09910490079B0C9AF9F7A3FA1290D0
:10BFC00000201090E3480D46784400680E9001214F
:10BFD00078104907084311990D9B890440180121E5
:10BFE000C90447183946029A0E98F9F77DFA324685
:10BFF000059BF9F77FFA02460B4629461098F9F798
:10C0000081FA064602913B4629460E9A1098F9F7A6
:10C0100079FA079B0C9AF9F76DFA3246029BF9F709
:10C0200063FA099B049AF9F76DFA0591129A0A903E
:10C030002B4610461946F9F765FA06460246C648E9
:10C040000F460B4606217844FEF79CFB32463B46E2
:10C050000091049010461946F9F754FA009B049A8F
:10C06000F9F750FA06460F462B461946129A1098D1
:10C07000F9F796F9059B0A9AF9F744FA32463B46D6
:10C08000F9F78EF9109A079104902B46104619463D
:10C09000F9F738FAB14E0022334609910290F9F7C8
:10C0A0007FF9079B049AF9F77BF9002007460246BF
:10C0B00033460091F9F718FA099B029AF9F714FA36
:10C0C000079B049AF9F716FA06460D913A46294657
:10C0D000009B1098F9F716FA07910C902B46304602
:10C0E000129A0D99F9F70EFA05460E463A46009B4C
:10C0F00005990A98F9F706FA33462A46F9F750F9EE
:10C1000002460B460746099107990C98F9F748F93A
:10C1100000250E462846079B0C9AF9F7E5F93A46A2
:10C12000099BF9F7E7F907460722099152078C4B5B
:10C1300031462846F9F7E6F907910090894A884B7D
:10C1400038460999F9F7DEF907460191864A874B87
:10C1500031462846F9F7D6F93A46019BF9F720F916
:10C16000834B7B440F9A9B181A685B68F9F718F9A0
:10C17000029009910398F9F7CDFA05910490099B73
:10C18000029A07990098F9F70BF97A4B7B440F9ABA
:10C190009B181A685B6817460393F9F701F9059B2A
:10C1A000049AF9F7FDF80E462846059B049AF9F71C
:10C1B0009BF93A46039BF9F797F9079B009AF9F721
:10C1C00093F9099B029AF9F795F902460B461999DA
:10C1D00000200C900F461898F9F794F902910490FA
:10C1E0003B460C9A19991898F9F77EF92A46334676
:10C1F000F9F788F9029B049AF9F7D2F809910E90A1
:10C200002A46334639460C98F9F77CF906460F461C
:10C21000099B0E9AF9F7C4F8574A0D46914220DB64
:10C220005242AA18024310D132463B46F9F75CF954
:10C2300004900391514A524B09990E98F9F7B0F8BE
:10C24000039B049AF9F720FB1ED20220FEF72AFB7B
:10C25000FEF704FB49004908E20FD20711431BB067
:10C26000F0BD6A00474B52089A420DD3464AAA18BD
:10C27000024300D0CBE532463B46F9F735F9099B3E
:10C280000E9AF9F701FBF5D96800002340082C4904
:10C290000393020D3D4B5218984223DD0120000507
:10C2A000521CD04042195000400D40183849794482
:10C2B000096813468C463749C1408B43120301215C
:10C2C000120B090551181422101AC1400391002DB8
:10C2D00001DA48420390624630463946F9F704F9DC
:10C2E00006460F4632463B4609990E98F9F758F82C
:10C2F00000252A46284B28460591F9F703F90791AE
:10C300000C90264A264B28460599F9F7FBF8009130
:10C31000029032463B4628460599F9F7E5F8099B15
:10C320000E9AF9F7E7F81F4A1F4BF9F7EBF8009B55
:10C33000029AF9F735F807460B460246099135E0AF
:10C3400001FCFFFF0000F03F8E9803007AB60B005F
:10C350006A070000AC070000D60600000000084095
:10C3600009C7EE3FFD033ADCF5015B14E02F3EBE4A
:10C37000AA0500007005000000009040FE822B65B9
:10C380004715973C00CC904000346F3F0000E03FE1
:10C39000C6040000FFFF0F00432EE63F396CA80CD7
:10C3A000615C20BEEF39FAFE422EE63F07990C98F9
:10C3B000F8F7F6FF05460E46079B0C9AF9F794F836
:10C3C0003A46099BF9F796F809912A4633460E90AA
:10C3D00010461946F9F796F8074602462F480B46CD
:10C3E000059105217844FEF7CDF93A46059BF9F70A
:10C3F00089F82A463346F9F77DF807460191284621
:10C400003146099B0E9AF9F77DF8099B0E9AF8F7C9
:10C41000C7FF012304910C9000229B073846019925
:10C42000F9F762F805910E903A4628463146019B8D
:10C43000F9F768F8059B0E9AF9F7CCF8049B0C9A6B
:10C44000F9F752F82A463346F9F74EF80022144B12
:10C45000F9F750F8064603980D46000541190915ED
:10C46000002912DC30462946039AF9F72BF9FEF72A
:10C4700043F9042801D1FEF7FBF930462946039A17
:10C48000F9F720F9064601E004E029180B46324688
:10C4900021460898F9F736F81BB0F0BD6803000094
:10C4A0000000F03FF0B58C46002510260521090755
:10C4B0008E620E4C08E067467F5DE760A768FF0765
:10C4C000FCD0E7681F706D1C8542F4DB0020074636
:10C4D00006E0E760A568ED07FCD0E5681D54401C48
:10C4E0009042F6D38E610020F0BD00000030014084
:10C4F00070B572B60124074DA40221462846F9F70B
:10C500009BFC002804D0224603492846F9F738FD51
:10C5100062B670BD00FC0008C00D0020F8B50646EC
:10C520000C46F9F7BFFA051E0F4600D00120014363
:10C5300049000B484908411AC90F0DD0002E01D0FF
:10C54000012100E000210C4361004908401AC00F9E
:10C5500002D10120FEF7A6F928463946F8BD0000B1
:10C560000000F07FF8B515460E460746002407E0A8
:10C570003819C0B200F008F8641C2870E4B26D1CD1
:10C58000B442F5D33046F8BD10B50446FBF7C4FFFE
:10C59000EE20FBF794FFFBF7F8FF2046FBF78FFF39
:10C5A000FBF7F3FFFBF7B8FFEF20FBF788FFFBF784
:10C5B000ECFF0020FBF756FF0446FBF7C8FF2046C0
:10C5C00010BD704770B50D460446FBF7A5FFEE2081
:10C5D000FBF775FFFBF7D9FF2046FBF770FFFBF772
:10C5E000D4FF2846FBF76BFFFBF7CFFFFBF7AFFF4E
:10C5F0000A20FEF7A0FA70BDF0B500251026052729
:10C600009C463F070B46BE620C4C06E0595DE1605C
:10C61000A168C907FCD0E1686D1C8542F6DB0020EB
:10C6200007E06146095CE160A168C907FCD0E168E8
:10C63000401C9042F5D3BE610020F0BD00300140A7
:10C640000000010203040005405C0000A05C04003F
:10C65000C06C0800805C0400E03F1E00E07D1E000E
:10C6600007A9022570889B880A00160001000600B1
:10C670000100020087008D002D001A3152001A338C
:10C680009A001A351D011A376B003B31BE003B334F
:10C690005E013B3596023B37000099599959EB51A1
:10C6A0008F421E45142E0080EB51F5283333E13ABA
:10C6B000703DE13AC235852BC2353333C235C235C0
:10C6C000AE47E13A5138A330513800000000000075
:10C6D00000000102030406070809030406080C1001
:10C6E00018203000000000010203040000000000D8
:10C6F000000000000000F03F000000000000F83FD4
:10C7000000000000000000000000004003B8E23F0D
:10C71000000000000000000006D0CF43EBFD4C3EBF
:10C72000033333333333E33FFFAB6FDBB66DDB3FB4
:10C730004D268F515555D53F01411DA96074D13FFC
:10C7400065DBC9934A86CD3FEF4E454A287ECA3FF6
:10C750003E5555555555C53F93BDBE166CC166BF78
:10C760002CDE25AF6A56113FF16BD2C541BDBBBE71
:10C77000D0A4BE726937663E0000000000000000D1
:10C78000A0C7000800000020680100006C5B0008E2
:10C79000F8C7000868010020B019000094A800083C
:10C7A0000124130704380D091E0805400826091046
:10C7B0004008560A131D043B08BE0516D8BC40109D
:10C7C0000852010336C84203585C121B0202BD1412
:10C7D00009010222815015339788979897598197BC
:10C7E000979097999785976981768249BD014529E8
:08C7F0004B92049220000000AE
:04000005080050C1DE
:00000001FF
